:100000000C940B030C9428030C9428030C942803E1
:100010000C9428030C9428030C9428030C94D834D3
:100020000C9428030C949B2A0C9477290C94332964
:100030000C94742A0C9428030C9428030C94280321
:100040000C9428030C9428030C9428030C94280384
:100050000C9428030C94502A0C9428030C94280325
:100060000C9428030C9428030C9428030C94280364
:100070000C9428030C9428030C9428030C94280354
:100080000C9428030C9428030C9428030C94280344
:100090000C9428030C9428030C9428030C94280334
:1000A0000C9428030C9428030C94280305010902DE
:1000B000A10185020901A1000509190129081500FE
:1000C0002501950875018102050109300931158165
:1000D000257F95027508810609381581257F9501D0
:1000E00075088106050C0A38021581257F95017572
:1000F000088106C0C005010980A101850319012AF4
:10010000B700150126B700950175108100C0050CD8
:100110000901A101850419012AA002150126A002E6
:10012000950175108100C00660FF0961A101096297
:10013000150026FF00952075088102096315002629
:10014000FF00952075089102C005010906A101056F
:100150000719E029E7150025019508750181029529
:1001600001750881010507190029FF150026FF0008
:100170009506750881000508190129051500250156
:10018000950575019102950175039101C0FD377ABE
:10019000585A000004E6D6B44602002101160000B9
:1001A00000742FE5A3E004AE01565D003D8889860A
:1001B000D3DC0AE842C324925842588FD8E75CA0A7
:1001C000D2616E26E888019A676C7887BC8D370902
:1001D000E9D5B739F4E81FA1588DAC1F8AD1B231E7
:1001E000310947F61CBFFFD9CCDFA7E34854EDF532
:1001F000D1109FD138BC29FCFF64C31636C878D40F
:10020000C49AAFCF36FD05742F195A7D842EA19C58
:10021000DF98E88625C64F0A607B98F5AD985CC7E5
:10022000B01AAB783D4FFF5809AF5A1590FECB502E
:10023000804F11BF6EBB6058C7CEA8ED87E4DF8C3E
:100240007F0461157CE3A2DB0E4AD173460C94E96E
:1002500067C597BE8EA3966DAAE8D2CD55A13ECDB7
:1002600058FBAAAEC8DD456C3999DDACB41B1C0B3C
:100270005ACBF899D933014C65216E2195CD6A2E60
:100280008B8E0DBF9F49F1ACBDFED4560F86817495
:1002900026F8EA663F54576D9571BD521BDD384D07
:1002A000AF4D46EAD53F9446DB882BABFDD4064CD8
:1002B00093CBD0EF48F0F93CE6F74C2EEFBE4CCF95
:1002C0002FDBAF761829DDB622EB6DB3EEB22DBC75
:1002D0003F41D54CC08FA535C599D8FB873F95AA1E
:1002E00039F24BF32B455C80F80AC85E972B3A1C19
:1002F000097D3057D1A8F88982D625FF4D2549219F
:100300005300000000CA4E3964D90BC0B80001F296
:1003100002AF090000730D16FBB1C467FB020000B9
:10032000000004595A01000100CD041B0F000F000A
:100330000002000200C9041B0F000F0000030001AF
:1003400000CE041B0F000F000004000200B3041BCA
:100350000F000FA60705000100CF041B0F000F00C0
:100360000006000200B5041B0F000F00000700028A
:1003700000CB041B0F000F000008000100D0041B7D
:100380000F000F000009000200B7041B0F000F81CF
:10039000070A000200B9041B0F000F81070B0002BF
:1003A00000BB041B0F000F81070C000200BD041BE3
:1003B0000F000F81070D000200BF041B0F000F810B
:1003C000070E000200C1041B0F000F81070F00027F
:1003D00000C3041B0F000F810710000200C5041B9F
:1003E0000F000F810711000200C7041B0F000F81CF
:1003F0000712000200D1041B0F000F0000130002BF
:1004000000D3041B0F000F000014000100D5041BD3
:100410000F000F00001500000000000707E01600A5
:1004200000290014000F0018003600370000002BD0
:100430000008000C00040012002D0000000000E184
:10044000001D001B0006001900000000000000E273
:1004500000E300E0002800000000000000000000B1
:1004600000000000002C0009001A0015001C0038D4
:1004700000330000000E001700110016000B0013DF
:100480000000000A00070010000D00050000000039
:10049000002A00E400E700E600000000000000522F
:1004A00000500051004F0028000000000009025BCE
:1004B00000030100A0FA0904000001030101000982
:1004C00021110100012244000705810308000109F0
:1004D0000401000203000000092111010001222291
:1004E000000705820320000107050303200001091E
:1004F0000402000103000000092111010001227B18
:10050000000705840320000112010002000000081A
:10051000EDFE00000001010203011C0376006900EA
:1005200061006C003A00660036003400630032005F
:1005300062003300630000000E0370006F0074005F
:100540006900340038000000180373006800690077
:100550006200610064006F0067006300610070006A
:100560000000040309040000000000000000000077
:10057000000000000000000000000000000000007B
:10058000000000000000000000007E0F00D4FFFF0C
:10059000FFC70000007800000000000000002A2BC8
:1005A0002800000000000000000000000000000023
:1005B0000029000000002C1E34202122243426278C
:1005C000252E362D3738271E1F20212223242526AD
:1005D0003333362E37381F0405060708090A0B0C7B
:1005E0000D0E0F101112131415161718191A1B1CC3
:1005F0001D2F3130232D350405060708090A0B0C81
:100600000D0E0F101112131415161718191A1B1CA2
:100610001D2F3130354C11241FBECFEFDAE0DEBF85
:10062000CDBF11E0A0E0B1E0EAE3FEE602C0059034
:100630000D92AC39B107D9F725E0ACE9B1E001C0C2
:100640001D92A435B207E1F70E94182B0C94F036E6
:100650000C940000482F209152059091090559E013
:10066000291302C080E0089530E0529FF001539FAB
:10067000F00D1124E65FFA4F8181681306C0808176
:10068000481303C085818111EECF2F5F3F4F277044
:10069000E7CFFC01AC014B5F5F4F8FEF91E32191FE
:1006A000822728E030E087FF09C0880F8927215082
:1006B0003109C9F7E417F50791F70895880FF7CFC7
:1006C000E8EDF0E080818E7F80831092E20010924E
:1006D000DA001092E100A0EEB0E08C9181608C9382
:1006E00080818F77808319BCA7EDB0E08C918E7FDD
:1006F0008C9380818F7E80831092F20408952091E4
:10070000E4003091E50095E6A9012091EC00822FEC
:10071000817020FF06C08091E80080FF06C080E065
:1007200008952091E80022FD1AC08091FF048823DB
:1007300089F0853089F08091EB0085FD0FC0209114
:10074000E4003091E50042175307F9F29150E1F6C9
:1007500084E0089582E0089583E0089581E008959B
:100760008091010587FF13C08091E80082FF06C0D9
:100770008091E8008B778093E80004C08091FF04AB
:100780008111F2CF08958091FF048823D9F38091DD
:10079000E80080FFF8CF8091E8008E77ECCF982FAB
:1007A0009093E900242F762F50E0891731F0709153
:1007B000EC002091ED005091F00021FD07C09F5FFB
:1007C000973071F78093E90081E008953091EB0054
:1007D0003E7F3093EB003091ED003D7F3093ED0094
:1007E0003091EB0031603093EB007093EC0020937C
:1007F000ED005093F0002091EE0027FDE0CF80E067
:100800000895B0E0A0E0E7E0F4E00C94FE35C8ED18
:10081000D0E088818F7E8883E7EDF0E08081816081
:10082000808384E082BF81E08093F20488818E7FA0
:10083000888302EE10E0F80110821092DA0081EE57
:10084000C82ED12CF601108288818F778883888109
:100850008068888388818F7D888319BC1092FF040B
:10086000109200051092FE041092FD0490EEE92E05
:10087000F12CF70180818B7F808388818160888360
:1008800042E060E080E00E94CF03F60180818E7F2D
:100890008083F8018081816080838081886080838B
:1008A000F70180818E7F8083888180618883CDB7C6
:1008B000DEB7E8E00C941A36FC01809107059091B0
:1008C000080586179707A0F06115710529F4909126
:1008D000E8009E779093E80090E06115710551F46F
:1008E000911108C08091E80082FF34C080E0089533
:1008F000BC01F2CF8091FF048823C1F18530C1F1A2
:100900008091E80083FD30C08091E80082FDEACF4D
:100910008091E80080FFE1CF8091F3002091F20008
:10092000382F6115710519F02830310558F091E024
:100930002830310509F090E02091E8002E772093CF
:10094000E800CBCF81918093F100615071092F5F56
:100950003F4FE7CF8091FF04882341F0853041F07D
:100960008091E80083FFBECF81E0089582E0089582
:1009700083E0089508958091F404089587E797E748
:10098000909301088093000888E19AE00FB6F894EC
:10099000A895809360000FBE90936000FFCF9C01EC
:1009A0004FB7F8948091EE049091EF04A091F00479
:1009B000B091F1044FBF821B930B08952FB7F894A9
:1009C0006091EE047091EF048091F0049091F10435
:1009D0002FBF08952FB7F8948091EE049091EF0403
:1009E000A091F004B091F1042FBF0895E0EAF1E086
:1009F0009191891303C0DF0111971C9291E0E63AAF
:100A0000F907B1F708959C01FC0132969FEF80E051
:100A10004191461751F09F3F19F4411101C0982FA1
:100A20008F5F8630A9F79F3F09F40895290F311D84
:100A300097FD3A95F90162830895A3E0B0E0E3E2FF
:100A4000F5E00C9404362091EB043091EC04281767
:100A50003907A1F09093EC048093EB04E091E90452
:100A6000F091EA04309751F024E029839B838A8334
:100A70000084F185E02DCE01019609952396E2E0F0
:100A80000C942036A3E0B0E0E8E4F5E00C940436E2
:100A90002091E7043091E80428173907A1F09093DA
:100AA000E8048093E704E091E904F091EA043097C8
:100AB00051F023E029839B838A830084F185E02D14
:100AC000CE01019609952396E2E00C942036E09140
:100AD000E904F091EA04309739F022E0DC012C932C
:100AE0000680F781E02D099508958091E50488231B
:100AF00059F0E091E904F091EA04309729F001906F
:100B0000F081E02D0995089580E008954115510583
:100B100011F0FA01099508950E94EA049C01909150
:100B2000DF048091E004982B21F03093DC042093C3
:100B3000DB049091E1048091E204982B21F0309342
:100B4000DA042093D9048DED94E00E94670508959E
:100B50008091D80480FF0CC060913C0170E07595D5
:100B60006795759567956115710549F1862F08950B
:100B700081FF06C060913C0170E075956795F3CFE9
:100B800060913C0182FD0BC09091D7049923A1F0A4
:100B900060913B0180913C01961738F0682F70E01E
:100BA0006038710500F38FE70895899FC001112413
:100BB00070E00E943F36F4CF61E070E0D7CF81E073
:100BC00008958091D8046091BB047091BC0480FFAB
:100BD00016C020913A01269FC001279F900D112435
:100BE000BC0176956795769567956038710508F034
:100BF00043C06115710509F441C0862F089581FF36
:100C00000BC020913A01269FC001279F900D11240F
:100C1000BC0176956795E9CF82FF09C080913A01C2
:100C20009B01829FB001839F700D1124DECF209124
:100C3000B2042223D1F29091390180913A01482FD8
:100C400050E0291748F0CB01849FB001859F700DBB
:100C5000949F700D1124C9CF289F90011124269FC5
:100C6000A001279F500D369F500D1124692F70E071
:100C7000CA010E942B36B9CF8FE7089581E008950D
:100C8000282F35EB2303C001112497FF04C080589F
:100C90009109892F089580589F4FFBCFCF93DF9301
:100CA000EC014091A7045091A8046091A9047091AF
:100CB000AA042FB7F8948091EE049091EF04A091CC
:100CC000F004B091F1042FBF841B950BA60BB70B5A
:100CD000843F9140A105B10518F58091A70490913A
:100CE000A804A091A904B091AA048093A3049093AE
:100CF000A404A093A504B093A60484EF91E0A0E01F
:100D0000B0E080939F049093A004A093A104B093BB
:100D1000A204D093AF04C093AE04DF91CF910895A5
:100D20000E94DE046093A3047093A4048093A5043E
:100D30009093A60482E390E0A0E0B0E0E2CFFC0153
:100D40008481862351F492819923B9F069238085A7
:100D500083FF05C081E061110FC080E00895892FF5
:100D60008F7092959F70982B862F8F7062956F7001
:100D7000682B81E09613F1CF089581E0FDCFDC016F
:100D80006091990480919A04962F891301C0089567
:100D9000292F30E0F901EE0FFF1FEF56FB4F408186
:100DA00051814A175B07A1F487E08A9FA0018B9FBE
:100DB000500D112440515C4F81E0FA018483961359
:100DC000E6CF2F5F3F4F2370332720939904089578
:100DD0002F5F3F4F922F9370D8CF1092EE03109257
:100DE000ED03E0EFF3E08581811102C014821682E9
:100DF000379684E0E832F807B1F7089524982C9AE2
:100E000008952C98249A089525982D9A0895B0E075
:100E1000A0E0EDE0F7E00C94FC358FEF9FEF44305D
:100E2000510508F469C04091A20341FB882780F96D
:100E300090E0880F991F42FB002700F910E0000F97
:100E4000111F000F111F802B912B40FBCC24C0F8E9
:100E5000D12C8C299D2943FB222720F9C22FE0E0C9
:100E6000DE2F53E0CC0FDD1F5A95E1F78C2B9D2B25
:100E700044FBAA27A0F9B0E0E4E0AA0FBB1FEA9563
:100E8000E1F78A2B9B2B45FBEE27E0F9F0E0A5E08C
:100E9000EE0FFF1FAA95E1F78E2B9F2B46FB222713
:100EA00020F930E0B6E0220F331FBA95E1F7822B2C
:100EB000932B47FB222720F930E03695322F22274B
:100EC00037952795822B932B2091A303322F3170D6
:100ED000F32EE82EF92A26952170B22EBB0CA82EEF
:100EE000BF28C501BB0CAA0BBB0BFB018083918300
:100EF000A283B38390E080E0CDB7DEB7EAE00C9444
:100F00001836E3EBF4E0848195812AE030E0B90102
:100F10000E942B3660933301868180933201828553
:100F200080933A0184858093390186859785B9013C
:100F30000E942B3660933101808980933001828931
:100F400080933C01848980933B0108958091B30490
:100F50009091B40490933601809335010895E9E5AA
:100F6000F2E090E080E064E778E24BE958E22AEEB4
:100F700037E2778366835187408733872287978755
:100F80008687019670968830910599F708958115A6
:100F90002CE7920741F420919D0430919E04232B6D
:100FA00011F490E080E0089580E00895F894E82F2F
:100FB000E295EF70F0E031A1282F2F7081E090E0F2
:100FC00001C0880F2A95EAF7982F9095932391A353
:100FD00092A1892B82A3789408950F931F938091F7
:100FE000E504882329F00E94DE041F910F910895E3
:100FF0000E94DE040091010210910202209103027E
:1010000030910402600F711F821F931FEECF811574
:1010100020E59207D0F5811540E4940708F08FC0D1
:10102000803E910520F58D3C910508F080C0883AFE
:10103000910578F4853A910508F070C081309105EA
:1010400019F1009709F184309105F0F490E080E007
:101050001BC0833C9105D0F7885AE82FF0E0EE0FD3
:10106000FF1FEB5AFE4F8081918194640895811592
:1010700050E2950708F0B8C0811561E0960708F0C6
:1010800058C0883E910510F70895803672E597079D
:1010900020F5803422E5920708F05BC0803242E5FB
:1010A000940708F04FC0811552E5950708F483C0F6
:1010B000282F2695269570E2279F90011124837092
:1010C00041E050E0BA0102C0660F771F8A95E2F74F
:1010D000CB01822B932B9D680895803A62E5960799
:1010E00060F4803872E5970708F449C08F7190E08A
:1010F000982F8827846F906A0895803C22E5920794
:1011000008F453C0803E42E5940708F09FCF982F23
:10111000882788279F71806F906A0895855AE82FE5
:10112000F0E0EE5AFE4F808190E090640895906563
:10113000089520E0392FB901682BCB0108959F70E5
:10114000906A08958F7190E0982F8827816F906A38
:101150000895282F26952695277070E2279F9001E5
:101160001124837041E050E0BA0102C0660F771F7E
:101170008A95E2F7CB01822B932B9C680895282F48
:1011800026952695277070E2279F90011124837081
:1011900041E050E0BA0102C0660F771F8A95E2F77E
:1011A000CB01822B932B9A6808958F7190E0982F32
:1011B0008827906208959C0195E0369527959A9529
:1011C000E1F72F7030E0322F2227482F4F7150E087
:1011D00084FF05C084E0440F551F8A95E1F7C901DB
:1011E000842B952B906908959F71E3CF8091DC014A
:1011F000882331F01092DC011092DB011092DA01A9
:101200000895CF93C82F8091A30382FF0CC08091D3
:10121000DC018C1741F00E94EA049093DB0180937B
:10122000DA01C093DC01CF9108959091DC01292F60
:10123000282361F0809589238093DC01882339F08D
:101240000E94EA049093DB018093DA01089590E014
:1012500080E0F8CF809590915305982390935305A3
:10126000089580959091C80398239093C80308959A
:101270009091C803892B8093C80308951092D101DF
:101280001092D0011092CF0108958091B5049091F1
:10129000B604892B89F00E94EA042091DA0130918A
:1012A000DB01AC01421B530B81E02091B50430916E
:1012B000B6044217530708F480E0817008959091B6
:1012C000CE01292F282321F0809589238093CE01F8
:1012D00008958091520590910905981301C00895D1
:1012E0008F5F8770FACF292F9A3078F5873068F5AD
:1012F00090E037E0239F800D911D1124682F6770C7
:1013000023E0969587952A95E1F7FC01EE0FFF1FE4
:10131000E80FF91FE655FE4F50E040E080E02191D4
:1013200030E0062E02C0369527950A94E2F7217028
:101330003327042E01C0220F0A94EAF7822B4F5F55
:101340005F4F4330510559F7089580E00895292FE4
:101350009A3098F5873088F590E037E0239F800D2C
:10136000911D1124282F277041E001C0440F2A95B8
:10137000EAF723E0969587952A95E1F7FC01EE0FB1
:10138000FF1FE80FF91FE655FE4F30E020E070E048
:101390005191DF011197CB01022E02C096958795DE
:1013A0000A94E2F7817081958527842385278C93A1
:1013B0002F5F3F4F2330310559F708958093120274
:1013C00008959091120221E030E0F90101C0EE0F82
:1013D0008A95EAF7D90102C0AA0FBB1F6A95E2F706
:1013E000EA2B01C0220F4A95EAF7892F8E23E813D2
:1013F00005C0292B822F0E94DE09089520952923FC
:10140000F9CF21E030E001C0220F8A95EAF720955C
:101410008091120282230E94DE0908959091D101E9
:10142000809589238093D101282F277069F489172B
:1014300059F09091A30392FF07C0869586958695F3
:101440000E94010A0E943E09089521E030E001C097
:10145000220F8A95EAF780911202822B0E94DE0900
:1014600008959091A30392FF10C098E0899F900186
:101470001124622B6093D1010E94250A0E94EA0484
:101480009093D0018093CF0108950E94250A08957A
:1014900080931102089592959F70963091F058F4C0
:1014A000925F9F70923058F4803F19F030F4883E7C
:1014B00030F481E008959A5FF4CF843FD1F380E067
:1014C0000895883EB0F3813FD1F7F3CF0F931F9378
:1014D000CF93DF93162F0FE2080FC82FD0E06623BB
:1014E00009F47BC08D3C41F40E94E1058195809315
:1014F000E0040E948C053EC08E3C19F40E94E10578
:10150000F6CF8F3C31F40E94E10581958093DF0492
:10151000F0CF803D19F40E94E105F8CF893D29F410
:101520000E94A8058093E104E4CF8A3D21F40E9443
:10153000A8058195F7CF8B3D31F40E94A8058195D0
:101540008093E204D6CF8C3D19F40E94A805F8CF11
:10155000083078F59E01215D310981E090E0AC0111
:1015600002C0440F551F2A95E2F78091DE04842BB8
:101570008093DE040330C0F440912B0250912C0282
:10158000C15DD10921E030E002C0220F331FCA95AE
:10159000E2F7C9019927112309F498C0842B952BF0
:1015A00090932C0280932B02DF91CF911F910F918A
:1015B00008958D3D31F48091D80481608093D804E2
:1015C00098CF8E3D21F48091D8048260F7CF8F3D73
:1015D00019F58091D8048460F1CF2091DF048D3C0F
:1015E00059F48091E00487FF0DC01092E0042111AE
:1015F0000BC01092B20408C08E3CA9F48091E004A4
:1016000018169CF32223A9F08091E1049091E20442
:10161000892B11F41092D704CE01815D91090897AE
:1016200008F4A8CF66CF8F3C49F427FFEBCF109288
:10163000DF048091E0048111E7CFDBCF803D19F416
:101640001216ACF3DFCF9091E104893D29F419160D
:10165000CCF61092E104D6CF8A3D19F497FFD2CF91
:10166000F8CF9091E2048B3D29F497FFCBCF1092F5
:10167000E204C8CF8C3D19F41916CCF3C3CF08305F
:1016800080F4AE01415D510981E090E001C0880F16
:101690004A95EAF780959091DE0489238093DE04D1
:1016A000B1CF8D3D31F48091D8048E7F8093D804E2
:1016B000A9CF8E3D21F48091D8048D7FF7CF8F3D47
:1016C00009F0A0CF8091D8048B7FF0CF80959095C2
:1016D0008423952365CF9C013A9521153F4150F510
:1016E000FC01EE27F170BC0166277270AC01442743
:1016F00054709C012227387094FF0EC080E1EF2BBC
:1017000009F480E0672B09F08062452B09F08064C2
:10171000232B89F08068089581E0EF2B09F480E0A5
:10172000672B09F08260452B09F08460232B19F0A8
:101730008860089580E008950F931F93CF93DF93FF
:101740008B01EA019091FF04943061F58093E900E8
:101750008FEF9091E800815095FD06C095ED9A9528
:10176000F1F700008111F5CF8091E80085FF1AC0E4
:101770000E947F03811111C08091E80085FD06C0A1
:101780008091E8008E778093E800F2CFF801819194
:101790008F018093F100219779F78091E8008E778F
:1017A0008093E800DF91CF911F910F91089543E05E
:1017B00050E0BC0184E00E949C0B089546E050E09C
:1017C000BC0184E00E949C0B0895CF93DF93EC0151
:1017D00048E050E0BC0181E00E949C0B88E0FE01E3
:1017E000A5EFB4E001900D928A95E1F7DF91CF91DA
:1017F0000895019708F40895EFE9FFE03197F1F7B4
:1018000000C00000F6CF8AE1815059F49FB7F894E8
:101810002091C4038091C503821313C080E09FBF51
:1018200008953FB7F8942091C5039091C4033FBF3A
:101830002913ECCFEFE9FFE03197F1F700C000008A
:10184000E3CF30E0F901EC55FC4F80812F5F3F4F33
:101850002F7133272093C403E2CF24982C9A85E07C
:101860008A95F1F7000083B18295817008952598DB
:101870002D9A85E08A95F1F7000083B185FB8827D2
:1018800080F90895CF93DF93C2E3D0E00E94370C34
:10189000811102C0209721F4CE01DF91CF910895EC
:1018A00085E08A95F1F700002197F0CFCF93DF9381
:1018B000EC010E94370C882311F0209721F4CE010F
:1018C000DF91CF91089585E08A95F1F70000219787
:1018D000F0CFEF92FF920F931F93CF93DF93E82EF9
:1018E00080916B008F7D80936B002D98259A0E94CC
:1018F000FE068FE891E00197F1F700C000000E941A
:1019000001070E94040780E197E20E94560C892B90
:10191000E9F1D0E0C0E011E0F12C01E0C7010C2EAC
:1019200002C0959587950A94E2F780FF3AC0102788
:101930000E94FE060E94420C892B41F182E390E056
:101940000E94560C892B11F12196C830D10531F730
:1019500080E58A95F1F7112339F10E94FE060E9475
:10196000420C892B99F082E390E00E94560C892B5F
:1019700069F090E59A95F1F70E94FE06C2E3D0E087
:101980000E942D0C8823C9F0209789F40E94040737
:101990000E94FE0680916B00806280936B0080E065
:1019A00033C00E940107C6CF0E940107D8CF25E0AF
:1019B0002A95F1F700002197E3CFCD2B39F382E38D
:1019C00090E00E94560C892B09F30E94420CC2E35E
:1019D000D0E0892BD9F20E942D0C811108C02097EC
:1019E000A9F285E08A95F1F700002197F4CFCD2B7D
:1019F00069F20E9404070E94FE0680916B008062DB
:101A000080936B000E94030CCDB7DEB7E6E00C9428
:101A10001C36B0E0A0E0EFE0FDE00C94FC357C016A
:101A20005B016A018091000201E010E08A3010F44D
:101A30000AE010E0C1E0D0E0B501C701F601099568
:101A4000811104C021960C171D072CF4CDB7DEB709
:101A5000EAE00C941836CC9F9001CD9F300D300DEC
:101A6000112490E080E045E34A95F1F700000196EB
:101A700082179307C1F7E0CFCF93C82F6FEF811183
:101A800061E184E290E00E94B4366FEFC1116DE233
:101A900085E290E00E94B4366FEFC1116CEA86E2F5
:101AA00090E00E94B436CF910895CF93DF93CCE6B7
:101AB000D3E060E0CE010E94B4362196C11584E0E7
:101AC000D807B9F7DF91CF9108951F93CF93DF9394
:101AD000122F8430E0F46A30D0F44730C0F4C42FC1
:101AE000D0E0CC0FDD1F9EE0699FC00DD11D1124F9
:101AF0009CE8899FC00DD11D1124632FCE018896CB
:101B00000E94B436612FCE0189960E94B436DF91CF
:101B1000CF911F91089584E290E00E949636813122
:101B200089F485E290E00E9496368D3259F486E27F
:101B300090E00E94963691E08C3A09F090E0892F6F
:101B40008170089580E0FCCF0F931F93CF93DF93B4
:101B5000843030F56A3020F5473010F5C42FD0E0DE
:101B6000CC0FDD1F2EE0629FC00DD11D11243CE87B
:101B7000839FC00DD11D1124CE0188960E949636F8
:101B8000082F10E0102F0027CE0189960E9496366C
:101B90009801282BC901DF91CF911F910F910895D2
:101BA00090E080E0F8CF462F20914302309144022C
:101BB000232B99F4703F39F4603F79F4809145020A
:101BC0009091460208957A3040F4673030F48430C2
:101BD00020F4672F0E94A40D089590E080E00895FE
:101BE000CF92DF92FF920F931F93CF93DF936C01FD
:101BF0000091120280911102082BC3E0D0E010E0A6
:101C0000FC2EC8010C2E02C0959587950A94E2F728
:101C100080FD0CC02197A0F7F12C8F2DDF91CF9183
:101C20001F910F91FF90DF90CF900895B6018C2FF8
:101C30000E94D30D0E940708019761F3EECFCF9366
:101C4000DF93EC010E94F00DBE010E94D30D0E94B3
:101C50000708DF91CF910895FC018481882371F0FA
:101C600087819085009729F00E9407080E944B0AFF
:101C70000895808191810E941F0EF8CF80E0089521
:101C8000A6E0B0E0E6E4FEE00C94033649835A8314
:101C900049815A819923A1F0222391F0CA010E941F
:101CA000F00D182F682F89819A810E94A7096981F8
:101CB0007A81812F0E94D30D2696E3E00C941F3683
:101CC000CA010E947309182FF2CFFC01262F8781C9
:101CD0009085009741F440815181628173818481B4
:101CE00095810E94400E08950F931F93CF93DF9329
:101CF00003EB14E0C8E5D2E0CE010E949636F8016D
:101D000061918F01681719F0CE010E94B4362196B7
:101D1000CC37F2E0DF0781F7DF91CF911F910F9170
:101D200008950F931F93CF93DF9303EB14E0C8E55F
:101D3000D2E0CE010E949636F80181938F01219660
:101D4000CC37F2E0DF07A9F7CFE2D3E0FE018591BF
:101D50009491009711F0FC0109952C96F4E0CB3298
:101D6000DF07A1F7DF91CF911F910F9108959B019C
:101D7000883070F49AE0899FB001112464587D4F37
:101D80004AE050E0C9010E94863690E080E0089564
:101D90008FEF9FEF0895AAE0B0E0E1EDFEE00C9434
:101DA00004369C0137552F3F310509F068F4BE0118
:101DB0006F5F7F4F0E94B70E892B31F489859A851A
:101DC0002A96E2E00C9420368091CB049091CC04CA
:101DD000F7CF9091A30392FB222720F9281779F0DF
:101DE00080FB92F99093A3036091A2037091A303E7
:101DF00084E090E00E94D23682E00E940E0A0895AC
:101E0000DA019C012E5F3F4FF90145915491F90190
:101E100025913491A217B30758F0FC0134968591AF
:101E200094910E9476360E94740E90E080E00895AE
:101E30008FEF9FEF0895DB01FC01329625913491DD
:101E40004217530758F0FC01349665917491A9012B
:101E5000CD010E94763690E080E008958FEF9FEFED
:101E60000895AAE0B0E0E7E3FFE00C94FC350AE255
:101E700013E08CE1E82E83E0F82E97E0B92E29E2FA
:101E8000C22E23E0D22EAA24A3944AE050E0B70148
:101E9000CE0101960E948636F8013896DF018B2D1F
:101EA0001D928A95E9F789819A81D80111969C93B0
:101EB0008E938F8112968C9312978D8113968C93AB
:101EC0001397888514968C931497898515968C930F
:101ED00015978B819C8117969C938E9316971896D5
:101EE0001C9218978A8587FF3CC01E961C921E92F2
:101EF0001D9780FF03C0D8011896AC9281FF04C0E3
:101F0000F80190859260908782FF07C0D8011896EB
:101F10009C911897946018969C9383FF04C0F801D5
:101F200090859860908784FF07C0D80118969C918F
:101F30001897906118969C9385FF04C0F8018085DE
:101F400080628087FAE0EF0EF11C015F1F4F8CE684
:101F5000E81683E0F80609F098CF2A96EAE00C9498
:101F60001836F801D686C586C4CFAAE0B0E0EBEB00
:101F7000FFE00C94FE35E9EDF2E080E5DF011D9213
:101F80008A95E9F7E0EFF3E088E3DF011D928A9597
:101F9000E9F789EDC82E82E0D82E7F010CEC12E023
:101FA000F701D182C0824AE050E0B801CE0101962B
:101FB0000E94863688E0FE013196D60101900D928E
:101FC0008A95E1F789859A85D70113969C938E931C
:101FD0001297BAE0CB0ED11CE7E0EE0EF11C065FC3
:101FE0001F4F0C31F3E01F07D9F62A96E8E00C9456
:101FF0001A36A4E0B0E0EFEFFFE00C940336409116
:10200000FC015091FD016091FE017091FF012FB71D
:10201000F8948091EE049091EF04A091F004B091B7
:10202000F1042FBF841B950BA60BB70B11E0843670
:102030009105A105B10570F10E94ED076E5F7F4F1C
:102040008F4F9F4F69837A838B839C83809112018A
:10205000909113018E509E4F4091110150E04530F8
:10206000510510F044E050E0BE016F5F7F4F0E94C9
:10207000763682E090E00E947E35182F882351F05A
:102080000E94DE046093FC017093FD018093FE01C9
:102090009093FF01812F2496E3E00C941F36EF927A
:1020A000FF921F93CF93DF9300D000D000D0CDB725
:1020B000DEB77B0190E080E00E947E35182F8823F8
:1020C00009F46AC04091040150E04115510511F036
:1020D00041E050E060910501709106016E507E4F25
:1020E000CE0106960E9476364091EE015091EF01A6
:1020F0006091F0017091F1012FB7F8948091EE0496
:102100009091EF04A091F004B091F1042FBF841BD3
:10211000950BA60BB70B84369105A105B10538F4D4
:1021200083EF91E00E9449039E818917A9F181E024
:1021300090E00E947E35882309F44EC040910C0146
:1021400050E04630510510F045E050E060910D013F
:1021500070910E016E507E4FCE0101960E94763630
:1021600083EF91E00E9449039E81891335C00E944C
:10217000DE046093EE017093EF018093F001909381
:10218000F10185E0FE013196A9EEB1E001900D92DA
:102190008A95E1F711E00BC085E0E3EFF1E0DE01A5
:1021A000119601900D928A95E1F71111EACF85E021
:1021B000E9EEF1E0D70101900D928A95E1F7812FC8
:1021C00026960FB6F894DEBF0FBECDBFDF91CF913C
:1021D0001F91FF90EF90089510E0E9CFAFE0B0E0DD
:1021E000E4EFF0E10C94F9358E010F5F1F4F8AE0A8
:1021F000F80111928A95E9F780E2C82E81E0D82E85
:10220000F12CE12CAA24A394B12C20E2822E21E00F
:10221000922EF60181916F018F3F09F442C0F8942C
:10222000E82FE295EF70F0E021A18F70A50102C0C8
:10223000440F551F8A95E2F7CA01922F982B91A35C
:1022400092A18095892382A3789400C0E9E1F1E00E
:10225000712C31E021912F3F09F48CC0A22FA2955F
:10226000AF70B0E090968C9190E02F7002C0959581
:1022700087952A95E2F780FD7DC0832F782A330F5A
:102280008E169F0639F7F601319780818F3F11F046
:102290000E94D60750EA5A95F1F7F801EE0DFF1D9E
:1022A00070828FEFE81AF80AE5E0EE16F10409F003
:1022B000B0CF4AE050E0B80185E092E00E94693674
:1022C000009741F02AE0F801A5E0B2E001900D92FC
:1022D0002A95E1F70091100210E0075C1D4F892B51
:1022E00009F44AC081E08093E1010E94EA049093DE
:1022F000E0018093DF01F12CE090E504EE2009F489
:1023000092C06E01FBE0CF0ED11C85E0F601119268
:102310008A95E9F7809100028A3008F051C04FE4B5
:1023200050E1B601C8010E94090D882309F46AC072
:1023300049EF5FE0B601C8010E94090D882309F446
:1023400061C01092000280910F0290E045E050E0E1
:10235000B601875C9D4F0E94693621E02093E80119
:10236000892B09F042C0E12C8E2D8F292F96EDE0AC
:102370000C94153680E082CFF090E101FF2009F443
:10238000BACF8091DF019091E0010E94CF040597C0
:1023900008F4B1CF45E050E065E072E0C8010E946A
:1023A0006936892B59F085E0E5E0F2E0D80101902B
:1023B0000D928A95E1F71092E1019ECFF12CFBCFAF
:1023C0008091E2019091E3010E94CF04843F91400B
:1023D00008F0A5CF8091E801882329F285E0F60175
:1023E00011928A95E9F71092E801A0910F02B0E0EE
:1023F000A75CBD4F85E0FE013B9601900D928A954A
:10240000E1F7B2CF809100028F3F31F08F5F809370
:1024100000028A3008F497CF0E94EA049093E30107
:102420008093E201D7CF85E0F801A3EFB1E00190FE
:102430000D928A95E1F783EF91E00E944903809322
:10244000F2018090F8019090F901A090FA01B0900B
:10245000FB018091E4019091E501A091E601B0912A
:10246000E70188169906AA06BB0609F47DCF80927B
:10247000E4019092E501A092E601B092E7010E948A
:10248000DE04861A970AA80AB90A8092010290927D
:102490000202A0920302B092040266CFCF93809111
:1024A000C803C0915305C82B8091DC018823E9F053
:1024B0008091B5049091B604892B29F00E944509BA
:1024C00081110E94F6088091DC01C82B20E080EA8F
:1024D00091E0FC013191CF0131112F5FF1E0863A9B
:1024E0009F07B9F721110E94F6088091AB048095EF
:1024F0008C239091AC04892B80939E0148E050E09E
:1025000062ED71E08EE991E00E946936892BA9F0B5
:1025100088E0EEE9F1E0A2EDB1E001900D928A953C
:10252000E1F7E091E904F091EA04309731F002809C
:10253000F381E02D8EE991E00995CF910895CF9335
:10254000DF93EC014A855B856E857F850E94860559
:102550008B810E942A098C810E9431090E944E12AF
:1025600086E0FE0111928A95E9F7DF91CF910895F7
:10257000CF93DF93EC018D8181FD14C082608D8348
:10258000809153059B81892B809353058C810E94F8
:1025900038090E944E12488559856E857F85CE0187
:1025A0000E9486051092E4041092E3048D8180FD60
:1025B00003C0CE010E949F12DF91CF9108958091B8
:1025C0003701877F8093370182E00E942A0980913A
:1025D000370184FF06C08F7E8093370182E00E941E
:1025E00038098091370185FF06C08F7D80933701C0
:1025F00080E20E9438090E944E120895CF931092F3
:10260000C803C6E0E0EAF1E0DF018C2F1D928A9555
:10261000E9F790E080E00E94420590E080E00E94AF
:102620001D05109253050E944E12EDEDF4E0DF01FE
:102630001D92CA95E9F71092B2041092D704109235
:10264000D8040E948C05CF910895AAE2B0E0EBE295
:10265000F3E10C94033681E095E02091F100DC0178
:102660002D93CD01B5E089309B07B9F78091020524
:10267000833009F472C0B8F4813009F449C0823063
:1026800009F4B3C08091E80083FF96C280910105F0
:10269000909102059A3008F08FC2E92FF0E0EE50D9
:1026A000F94C0C9453368A3009F48EC08B3009F4FF
:1026B00071C0893039F780910105813219F7809115
:1026C000050590910605009711F00297D9F68091C3
:1026D000E800877F8093E8008091E80082FF38C09F
:1026E0009091F3008091F200029731F48091F10013
:1026F000813011F0863021F48091F1008093F40450
:102700008091E8008B778093E8000E94B003BACFF5
:1027100080910105813A09F0B5CF8091E800877F6B
:102720008093E8008091050590910605892B61F45E
:1027300068E085EF94E070E00E945C048091E8001E
:102740008B778093E8009ECF60E090E080E0F3CF4D
:102750008091FF048111C0CF95CF80910105813A0E
:1027600009F090CF8091050590910605892B09F01D
:1027700089CF8091E800877F8093E8008091E8000E
:1027800080FFFCCF80913D018093F1008091E800B3
:102790008E77B9CF80910105813209F073CF809196
:1027A000050590910605892B09F06CCF8091E80012
:1027B000877F8093E8000E94B00380910305809397
:1027C0003D010E94FE125ECF80910105813209F029
:1027D00059CF8091E800877F8093E8000E94B00382
:1027E000809104058093F3044DCF80910105813AD7
:1027F00009F048CF8091E800877F8093E8008091BE
:10280000E80080FFFCCF8091F304BECF803899F0C0
:10281000823809F0D1C1809105058F70873008F0AA
:10282000CBC18093E9008091EB0085FB882780F97C
:102830001092E90006C08091FD049091FE04911170
:1028400082609091E800977F9093E8008093F10078
:102850001092F1008091E8008E77AAC1882309F4D4
:1028600098C1823009F0A8C18091030581119BC1F4
:10287000809105058F702FEF280F263008F09CC13E
:102880008093E9002091EB0020FF8DC1933031F45B
:102890008091EB0080628093EB0085C19091EB000A
:1028A00090619093EB0021E030E001C0220F8A9507
:1028B000EAF72093EA001092EA008091EB0088602A
:1028C000EACF811179C1109103051F778091E30050
:1028D0008078812B8093E3008091E800877F80934C
:1028E000E8000E94B0038091E80080FFFCCF809157
:1028F000E30080688093E30082E0111183E080931D
:10290000FF045AC18058823008F056C12091030557
:10291000309104052C3DE3E03E07A1F583E08A8376
:102920008AE289834FB7F894DE01139620E03EE0F7
:1029300051E2E32FF0E050935700E49120FF03C0F1
:10294000E295EF703F5FEF708E2F90E0EA30C0F0BD
:10295000C7968D939D932F5F243159F74FBF809178
:10296000E800877F8093E8006AE270E0CE0101967C
:102970000E945C048091E8008B778093E8001CC182
:10298000C096E7CF8091050590910605432F552706
:102990004330510509F44AC078F54130510509F436
:1029A00085C08BE590E0EDEAF4E04230510509F096
:1029B00003C12091E800277F2093E80020910705BC
:1029C000309108058217930708F49C0140E0211517
:1029D000310509F070C041116EC08091E80082FDA0
:1029E000C9CF8091FF04882329F2853019F28091A4
:1029F000E80083FFF2CFBECF4132510509F447C052
:102A00004232510509F0D8C08330910508F0D4C096
:102A1000FC01EE0FFF1FE057FE4F0190F081E02D0B
:102A200083579E4FDC018C9190E01DC033272130ED
:102A30003105E9F02115310579F022303105F9F041
:102A40002330310509F0B8C0EAE1F5E0E4918E2FBA
:102A500090E0EAE1F5E007C0E2E6F5E0E4918E2FD0
:102A600090E0E2E6F5E0009709F4A6C0A2CFE8E422
:102A7000F5E0E4918E2F90E0E8E4F5E0F4CFE8E3B0
:102A8000F5E0E4918E2F90E0E8E3F5E0ECCF8330C1
:102A9000910508F091C0880F991FFC01EA56FE4F7E
:102AA0000190F081E02D89E090E083CF82E190E019
:102AB000E8E0F5E07ECF8091FF04882309F45ACF47
:102AC000853009F457CF8091E80083FD53CF809182
:102AD000E80082FD82CF8091E80080FF78CF90915E
:102AE000F3008091F2002115310519F0883091052D
:102AF00050F041E0089709F040E08091E8008E77BF
:102B00008093E80064CF44914093F10031962150C6
:102B100031090196E8CF803809F04EC08091E80075
:102B2000877F8093E800809100058093F10092CE2A
:102B3000811142C0109103051230F0F58091E80038
:102B4000877F8093E800109300050E94B003112353
:102B500011F084E005C08091E30087FDFACF81E0A9
:102B60008093FF0442E061EC81E00E94CF0342E2E7
:102B700061EC84E00E94CF0342E261EC82E00E94BB
:102B8000CF0342E260EC83E00E94CF038091FF0418
:102B900013C080910305813079F481E0933009F00E
:102BA00080E08093FE041092E9008091E800877F26
:102BB0008093E8000E94B0038091E80083FF0AC080
:102BC0008091E800877F8093E8008091EB0080622D
:102BD0008093EB00AA96E3E00C941F36E3EBF4E05D
:102BE000128E138E8FEA90E09183808325E0248FEC
:102BF00088E893E1938382838AE090E095838483DD
:102C000044E150E05783468348E050E051874087D5
:102C1000938782876EE170E07587648797878687E0
:102C200080E590E0918B808B538B428B48E250E0A3
:102C3000558B448B42E350E0578B468B48EC50E079
:102C4000518F408F158E178E168E91A380A322A3CD
:102C50000E94740E0E94FE121092A3031092A2030F
:102C6000E3EAF3E08081846080836091A203709145
:102C7000A30384E090E00E94D2360E94910E089552
:102C8000AEE1B0E0E6E4F6E10C94FC35E0909D04A2
:102C9000F0909E0481E090E090939E0480939D04C8
:102CA000B12C81E2C82E84E0D82EA12C1DC0402F6B
:102CB00021E030E0B11008C0F801EE0FFF1FEC0D6D
:102CC000FD1D859194919C016A2D8B2D0E94650DAF
:102CD0000F5F1F4F0730110551F7A3948EE0C80E08
:102CE000D11CEAE0AE1619F010E000E0E0CFB3949A
:102CF000F4E0BF12D6CF0E94EE151A8219821C8210
:102D00001B821E821D8218861F8288EC90E09A87A3
:102D100089870CE712E04AE050E0B801CE01019645
:102D20000E94D836065F1F4F0C3C82E0180799F7C7
:102D30006E01EBE0CE0ED11C8AE0F60111928A956D
:102D4000E9F74AE050E0B801C6010E94D836065FB4
:102D50001F4F0C31F3E01F07A1F76E0185E1C80E8C
:102D6000D11C8AE0F60111928A95E9F78FEF9FEF67
:102D70009A8F898F87E08E8F4AE050E0B801C601B4
:102D80000E94D836065F1F4F0C36F3E01F07A1F7ED
:102D9000F0929E04E0929D046E96EAE00C94183640
:102DA00080E00E943C0D60E087E290E00E94B43633
:102DB0000E9440160E94550D81E00E943C0D08952E
:102DC000CF92DF92EF92FF928FEF9FEF4430510549
:102DD00008F46CC0FB01C080D180E280F3800E94C7
:102DE000FE128091A203C0FA80F9B701A601769580
:102DF00067955795479540FB81F9B701A60122E0F9
:102E000076956795579547952A95D1F740FB82F9B6
:102E1000B701A60133E076956795579547953A95A2
:102E2000D1F740FB83F9B701A601E4E076956795F9
:102E300057954795EA95D1F740FB84F9B701A6016C
:102E4000F5E07695679557954795FA95D1F740FB4C
:102E500085F9B701A601A6E0769567955795479540
:102E6000AA95D1F740FB86F9B701A601B7E07695A0
:102E7000679557954795BA95D1F740FB87F98093A9
:102E8000A2038091A303D0FA80F9D1FACC24C0F830
:102E9000C0FA81F98093A3036091A2037091A30308
:102EA00084E090E00E94D23690E080E0FF90EF90C6
:102EB000DF90CF9008950E94FE122FEF84E39CE0F4
:102EC000215080409040E1F700C0000088E19AE086
:102ED0000FB6F894A895809360000FBE90936000A1
:102EE000FFCF882321F00E942A090E944E120895E4
:102EF000882339F090915305982B909353050E94A5
:102F00004E120895882321F00E9431090E944E122A
:102F10000895882321F00E9438090E944E120895D6
:102F2000882381F19CEF980F913A28F40E94F604CF
:102F30000E944E12089590E2980F983050F48770D6
:102F400091E001C0990F8A95EAF7892F0E94310913
:102F5000EFCF9BE5980F933028F490E080E00E943B
:102F60004205089598E5980F9B3128F490E080E0A1
:102F70000E941D05089593E3980F933118F460E0C3
:102F80000E94660A0895FF920F931F93CF93DF93D9
:102F9000F82E0091B0041091B1040115110509F447
:102FA00049C01092AF041092AE041092AB0410927C
:102FB000AC04D8011696CD91DC919E013A9521156D
:102FC0003F4108F4D07ED1E0C11101C0D0E0D8016A
:102FD0001996ED91FC911A97309731F01B966D91EF
:102FE0007C9180E00995D823DD2339F08CEF8C0F9C
:102FF000813A30F58C2F0E94F604FF2099F0E09181
:10300000B004F091B104808584FD0CC08091AD04C2
:10301000882341F0808191819C01215031092F3317
:103020003E47A0F00E944E121092B1041092B004DC
:103030001092AD04C801CDB7DEB7E5E00C941D36A3
:103040000E944E128C2F0E949017D7CF0E944E06DE
:10305000E9CFCF93DF93EC010E949017CE010E943D
:103060006B0B9E01205E31092830310510F0CD2B0D
:1030700029F40E948217DF91CF9108950E94711761
:10308000FACFCF93C82F8823A1F08CEF8C0F813A11
:1030900090F4E0EAF1E08191C817E9F181E0E63AC5
:1030A000F807C9F76C2F8EE991E00E9403050E9492
:1030B0004E12CF91089580E28C0F883048F4C7708B
:1030C00081E001C0880FCA95EAF70E943809EFCF66
:1030D000EBE5EC0FE33040F4F0E0EE5AFE4F808178
:1030E00090E00E944205E5CFE8E5EC0FEB3150F4AB
:1030F000F0E0EE0FFF1FEB5AFE4F808191810E949E
:103100001D05D7CF83E38C0F833198F661E08C2FB8
:103110000E94660ACECF8C2F0E94F6040E944E12A7
:10312000C1CF1F93CF93DF93182FEB010E9441185B
:10313000209739F4812F0E949017DF91CF911F9132
:1031400008958FE99FE00197F1F700C000002197F3
:10315000EFCF6091D3047091D404893321F0609152
:10316000D1047091D2040E9491180895B0E0A0E0BB
:10317000ECEBF8E10C94FC35EC018AE0A82E2881F8
:10318000222309F49EC0213009F043C08981813097
:1031900049F48E010E5F1F4F8A810E94A918E80131
:1031A0002196EDCF823039F48E010E5F1F4F8A8158
:1031B0000E944118F4CF833039F48E010E5F1F4F07
:1031C0008A810E949017EBCF843011F02196E8CFCE
:1031D0002A81229690E080E0AE014F5F5F4F20533E
:1031E000330B2A30310550F00097D1F2EFE9FFE0C0
:1031F0003197F1F700C000000197F6CFA89EB0010B
:10320000A99E700D1124C901860F971F2981EA011B
:10321000E3CFE22FF0E0EA56FA4FB490822F869582
:103220008695869590E0FC01EA57FA4FE490277066
:10323000F12C022E02C0F594E7940A94E2F7F1E033
:10324000EF22FF24FC01EA58FA4FC490D12C022E41
:1032500002C0D594C7940A94E2F731E0C322DD247A
:10326000FC01EA59FA4F049110E002C01595079548
:103270002A95E2F701701127E114F10419F081EEAB
:103280000E944118C114D10419F086EE0E94411821
:1032900070E060E08B2D0E949118C114D10419F0E8
:1032A00086EE0E949017E114F10419F081EE0E945D
:1032B00090170115110509F473CF8CE20E94A9182B
:1032C0006FCFCDB7DEB7EAE00C941836CF93DF931B
:1032D000EC010E946B0B9E01205E31092830310504
:1032E00010F0209741F40E9489178C2F0E944118FA
:1032F000DF91CF9108950E947817F7CF662329F0C8
:10330000209153052260209353059C0130522115D2
:10331000304308F499270E9466190895B0E0A0E0B0
:10332000E4E9F9E10C94FE356C018B01E42E809107
:10333000370182FF87C0C091EB03D091EC03CC151D
:10334000DD0521F0C114D10409F07CC08091370162
:103350008B7F8093370181FD6EC08091E90390914E
:10336000EA03A801481B590B81E0209135013091F7
:1033700036014217530708F480E08170F82E8091DF
:103380003701F0FA81F980933701FE0183E0F69569
:10339000E7958A95E1F7EE71FF27E753FC4F20810F
:1033A0003181AE014F70552781E090E002C0880F57
:1033B000991F4A95E2F7FF2009F43FC0822B932B17
:1033C000918380838091C80381FF08C08091370179
:1033D00080618093370182E00E9431098091C803A7
:1033E00085FF08C08091370180628093370180E2B9
:1033F0000E9431096F2DCE010E947E19EE2031F01E
:103400008091CE0485FF02C086FF30C08091D10438
:103410009091D2040E94F90B8091EB039091EC0300
:103420009C0130522115304308F499270E94291835
:103430000E94DF1217C081E0A0CF80959095822373
:103440009323BECFC601905281159043A0F4C601CC
:1034500099270E9429188091EB039091EC038C1519
:103460009D0531F31093EA030093E903CDB7DEB76E
:10347000E8E00C941A36C601ECCFA8E0B0E0E3E433
:10348000FAE10C94F4357C01DC0114968C918823CC
:1034900009F464C161E0C7010E94650E8C01F70167
:1034A0008581882331F18091E3049091E4040097B1
:1034B00001F108171907E9F0FC01FF27887F992718
:1034C000892B09F069C0A4E0EE0FFF1FAA95E1F770
:1034D000E75AFD4F85818460858311830083CF0186
:1034E0000E94B8121092530561E0C7010E94650E58
:1034F0008C01D70115968C91882309F4BBC0C801B3
:1035000097578038910508F0E8C0D02EBFE0B0177B
:1035100008F415C18FEF93E00E94963681110FC118
:103520000CE613E0D1103BC0F4E04F2E9E012F5F5C
:103530003F4F390133243A94D301E42D1D92EA958B
:10354000E9F76801FFEFCF1ADF0AC8010E9496363B
:103550008983882309F4F3C08130D1F4580122E033
:10356000A20EB11CC6010E949636582E8A8388236B
:1035700009F4E5C08FEF850D8330F8F4680133E07E
:10358000C30ED11CC5010E9496368B838823F1F1AE
:10359000C3010E94B6183AC0F0E0E0E09BCF0115ED
:1035A000E4E01E0709F4CBC0C8010E9496368111E1
:1035B00001C0DA940F5F1F4FB5CF8BEF850D8330BD
:1035C00068F5480143E0840E911CC5010E949636BF
:1035D0008B8364018823D1F0680154E0C50ED11CAF
:1035E000C4010E9496368C83882381F08B819C8154
:1035F0008130AFEF9A0710F0982F8827B6E05B165E
:1036000039F0E7E05E1639F00E946328860194CF16
:103610000E943E28FBCF0E94C527F8CFF4E0650149
:103620005F12F4CFC5010E949636B82E680124E0DF
:10363000C20ED11CC80103960E949636BB2009F425
:103640007EC0882309F47BC0482F4150550B349E1F
:10365000C001359E900D1124AB2DA150BB0B8A0FDC
:103660009B1F019798F2EFE9FFE03197F1F700C057
:103670000000F7CF680127E5D21A3FEFC316D10447
:1036800009F058F56FE472E08C2D0E94B70E892B7B
:1036900021F5C60174E0880F991F7A95E1F7FC01C6
:1036A000E75AFD4F22812130A1F520914F02309140
:1036B0005002232B91F02091510230915202232B82
:1036C00061F0209153023091540240915502509183
:1036D0005602242B352B232B21F1D70115965C9014
:1036E000552009F43FC00E35BCE71B0729F10F3503
:1036F000ECE71E0741F00D35FCE71F0799F58091B7
:1037000000018823C9F01092000180E00E94C317D5
:1037100016C0223011F72091530230915402232B0E
:10372000E1F2FC01E25AFD4F20812E7F2083875A6F
:103730009D4F0E94B812D1CF81E08093000180910B
:10374000D101877059F0F7018581882339F0809184
:10375000A30382FF03C082E00E940E0A2896E2E1E2
:103760000C94103680910001882309F4B9C4380103
:1037700020EE621A71084090DC018091CE01482A47
:103780008091C803482A38E06316710408F087C0A6
:1037900098012770332781E090E001C0880F2A95B7
:1037A000EAF7552009F478C0482AD7018D919C91F9
:1037B0000E94730921E030E0190102C0220C331C81
:1037C0008A95E2F7E091B004F091B104FE83ED83B5
:1037D0002091A6013091A70138872F836AE2C62E77
:1037E00063E0D62EB12CA12CB8E0AB16B10409F4DD
:1037F000D8C4411005C0D60112968C9181118BC09E
:10380000F601838190E082219321892B09F483C002
:103810008085982F977009F487E0F8E06F1671049F
:1038200008F057C0552009F450C086958170882350
:1038300009F471C0D6018D909C900815190519F4F2
:10384000552009F468C0ED81FE81EC15FD0509F4F1
:1038500062C0D6011D96ED91FC91309721F08081D8
:10386000882309F458C0642DC6010E949F0688234E
:1038700009F451C00815190509F038C501151105DD
:1038800009F439C5511039C5EF81F8858E169F06A8
:1038900009F041C0512C31C58095482286CF552072
:1038A00009F468C41093A7010093A6010E94DE04E6
:1038B0006093A7047093A8048093A9049093AA042A
:1038C0001092AF041092AE0470CF82FB882780F96B
:1038D000AECF552001F18170AACF0E94901732C55A
:1038E0000497813A910558F46C2D8EE991E00E947D
:1038F0000305552009F4F4C30E944E1220CF0E9404
:103900004E128FE39CE90197F1F700C000008C2D67
:103910000E944118EECF9FEFA91AB90AAFE0CA0E74
:10392000D11C62CFDC012D913C910217130709F0E5
:10393000D1C35110D1C31092AD0480E00E94C317CF
:10394000CFC3902F812F11C4F90144855585668519
:103950007785C9010E948605D60115968C9181FF55
:1039600034C4C6010E949F128091E3049091E40444
:103970000817190709F029C41092E4041092E3040F
:1039800024C490913701892F8E7F90FF81608093AE
:1039900037010E94DF1244C4809137018E7FF7CF38
:1039A000809137018F7E013E110531F0053E1105F2
:1039B000E9F4809137018F7D809337018091370141
:1039C00080FF19C0D70115968C910832110520F59A
:1039D0000E31110508F071C00430110578F5882307
:1039E00051F01092EC031092EB0305C0C801905205
:1039F0008115904318F7F70185810737FCE71F070A
:103A000009F4D0C008372CE7120709F013C4882343
:103A100009F4D7C082E0C9C00933110558F40D324A
:103A2000110518F40B321105D1F69091CE0492FDD8
:103A3000D6CF08C004361105C1F3D1CF9091CE0482
:103A400094FDCDCF882309F4A6C08091DC0190912C
:103A5000C803892B8D7FB1F11092EC031092EB0318
:103A60008091CE0481FD2EC0F80143E0F695E795E4
:103A70004A95E1F7EE71FF27E753FC4F98012F704D
:103A8000332781E090E002C0880F991F2A95E2F762
:103A90008095909520813181822393239183808327
:103AA00060E0C8010E947E198091DC018D7F0E9438
:103AB000010982E00E940E0A42CE9091CE0493FD4D
:103AC0008ECFC0CF89E0F701A1E2B2E001900D9264
:103AD0008A95E1F710922402109223028091EB0361
:103AE0009091EC0308171907D1F52091CE0425FF1A
:103AF00036C03091370131FF02C026FF30C020911F
:103B0000E9033091EA035601A21AB30AB7010E94F1
:103B1000CB0EA816B90618F58091C80381FF08C01E
:103B20008091370180618093370182E00E943109E2
:103B30008091C80385FF08C080913701806280931F
:103B4000370180E20E94310960913701669561700A
:103B50008091EB039091EC030E947E19F0CD80914F
:103B6000DC019091C803982B2091370191FB21F93A
:103B7000209337018D7F0E9401091093EC0300937D
:103B8000EB03D092EA03C092E9038091370184608D
:103B9000809337018ECF970140E0B601C8010E94A3
:103BA0008E19CDCD882349F081E00E94250A43E09B
:103BB00062E081E00E94E109C2CD81E00E94010A39
:103BC000F6CF82E0FBCF0B353CE7130749F10C350C
:103BD0004CE71407D9F00A351C4709F040C381E0CF
:103BE0001CC00E94FE128FEF94E3ACE08150904025
:103BF000A040E1F700C000000E94BE046FEF7FEF1D
:103C000090E080E00E94D2360E945B178091A3036F
:103C100082FB882780F991E089270E94E90E1FC363
:103C200080E0FBCFF701858100811181882369F055
:103C3000C8010E94F00DD82E682FC8010E94A70964
:103C4000B8018D2D0E94D30D11C3C8010E947309C4
:103C5000D82EF6CFE02FEF70DE2E802F807F19F068
:103C6000D29490EFD922CC20A9F0DD2059F080E247
:103C7000810F883010F0111107C08D2D0E94380976
:103C80000E944E12812F3FC080915305D82AD092B6
:103C90005305F6CF812F0E949017DD20B1F180E20D
:103CA000810F883010F0111104C08D2D0E94310950
:103CB00003C08D2D0E942A090E944E1226C0F02FAB
:103CC000FF70DF2E802F807F803219F0D29480EF3A
:103CD000D822112351F0113009F499C0CC2009F4F5
:103CE000A5C0BB2009F449C0CDCF8091A30382FDBC
:103CF00040C0CC20C1F1DD2029F08D2D0E94380973
:103D00000E944E1280E00E944118A92DA850BB0BC2
:103D1000149710F40E947505812F902F0E944B0A72
:103D20008111B8C11092A9011092A801AA20B1F086
:103D30008091D10180FD12C0D70115961C92869505
:103D4000869586950E94250AC7010E943D1A80919A
:103D5000D1018695869586950E94010A60E0C7018B
:103D60000E94650EFBCC80E00E949017DD2069F276
:103D70009CCFCC2091F1B11004C08D2D0E948917E9
:103D8000C4CF21E0B21211C08090DC018D2D8821BA
:103D9000D81609F4BACF0E94EA049093DB0180930D
:103DA000DA01D828D092DC01B0CF8091CF048230E4
:103DB00008F4ABCFB812A9CF8D2D0E9489178D2D95
:103DC0000E9415098091CE019D2D9823D91609F4E2
:103DD0009CCFD82AD092CE0198CFB1100AC08D2D99
:103DE0000E9482178D2D0E9415098D2D0E945F095A
:103DF0008CCF8091CF04823008F487CF31E0B312AA
:103E000084CF8091C8038D2109F47FCFE8CF8091C2
:103E1000D504CC2021F08B1508F477CFAECFB8169F
:103E200008F073CF8D2D0E9482176FCFBB20D1F386
:103E30008091D3049091D404193321F08091D1045E
:103E40009091D2040E94F90B812F0E9490175DCFB0
:103E5000802F86958695837069F0813009F055CF63
:103E6000812F902F9370C11002C080E090E00E94DB
:103E70001D054BCF812F902F9370C11002C080E0A1
:103E800090E00E94420541CF6C2D812F0E94660A6E
:103E90003CCF802F837091F5C11037CF412F4295D1
:103EA00046954770440F440F812F8F70042E01C038
:103EB000880F0A94EAF7212F207114FF07C02FE022
:103EC00030E001C0220F4A95EAF72095302F369551
:103ED00036953370323069F050F440911102313030
:103EE00029F0822B84230E94480A0FCF842B822B37
:103EF000FACF282B809111028227F5CF8695CC200E
:103F000011F0802F8170882309F4FFCE412F429554
:103F100046954770440F440F812F8F70042E01C0C7
:103F2000880F0A94EAF7212F207114FF07C02FE0B1
:103F300030E001C0220F4A95EAF72095302F3695E0
:103F400036953370323069F050F4409112023130BE
:103F500029F0822B84230E94DE09D7CE842B822B6A
:103F6000FACF282B809112028227F5CF402F4F7075
:103F7000D42ECC2029F0842F0E94250A812FFECE3A
:103F8000812F0E9482178D2D0E94010ABECE123F02
:103F900089F160F4103FB9F0113F81F0CC2009F4B1
:103FA00074C0B1106FCE802F8F7128C0133F49F1BC
:103FB000143FA1F78091A30382FD2FC0802F8F7142
:103FC000CC2011F31BC08091D504CC2079F0B81619
:103FD00008F09BCE202F2F7181E090E001C0880F68
:103FE0002A95EAF7909112028927B5CF8B1508F42C
:103FF0008CCEF0CF802F8F71C110C6CF0E94250AC2
:1040000084CE80E0CC2009F4A6CF81E0902F9F7170
:1040100001C0880F9A95EAF79ECF8091CF04823035
:1040200008F1CC20A9F09091D1019770943041F41F
:104030000E943E09802F8F710E94010AA12C65CE3B
:1040400063E0B816D8F7802F8F710E94310AF6CF3F
:10405000B81620F00E943E0964E0F5CF81E00E948E
:104060000E0AECCFCC2031F063E0802F8F710E94DC
:10407000310A4BCE81E00E940E0A51E05B1508F038
:1040800044CE82E00E940E0A40CEB110D1CE802FE5
:104090008F717ACFCC2019F0B11044CE47CEB11039
:1040A00041CE20E0F701408151816281738184819A
:1040B00095810E94400E8091D00483FF33CE809181
:1040C000A8019091A901029709F02CCE812F0E949E
:1040D000A91828CE552021F0FC01808585FF2DCC24
:1040E000C80197558F3F910511F008F06EC0C801C7
:1040F000887F9927892B09F022CBF801FF2754E00C
:10410000EE0FFF1F5A95E1F79F01275A3D4F6901B6
:10411000D70115968C91E25AFD4F908180FB90F962
:104120009083882309F410CC0E94EA049093200223
:1041300080931F02F60182818F5F828380915305F5
:104140009091C803892B83838091DC01848346810D
:10415000578166857785C6010E948605D60115962A
:104160008C9181FFEECB90E080E09093E30480930C
:10417000E4042BC08091A6019091A70108171907AC
:1041800081F41092A7011092A6011092A704109238
:10419000A8041092A9041092AA041092AF041092DD
:1041A000AE048091B0049091B104009709F498CFC7
:1041B000E8E06E16710408F0B5CB642D0E949F06EE
:1041C000811103C081E00E94C3178091CE0480FF5B
:1041D00012CC0E94EA046C01F7018581882309F45E
:1041E000DFCB8091370182FF08C021E232E040E05E
:1041F000B60190E080E00E948E190431FCE71F07B1
:1042000009F4CACB05312CE7120709F4BACB033104
:104210003CE7130729F480913701816080933701CF
:10422000C80190528115904308F0C8CB1092EC035E
:104230001092EB03D70115968C91882381F00330FF
:10424000BCE71B0709F4DACC08F0BDCC0115FCE78C
:104250001F0709F4C6CC01301C4709F4D5CCD7019F
:1042600017968D919C91009709F4DCCC0E94070869
:10427000182F092FD7011596CC9015971696BC903C
:10428000B2943FE0B3228091D101877001F1AC2C50
:10429000CC20F1F0892F807F803461F080E2810FA3
:1042A0008830A8F0892F807E803221F4123078F097
:1042B000BB2069F08091A30382FF09C082E00E94C5
:1042C0000E0A8091D1018770AA24A3948111A12C98
:1042D000902E92942FE09222BBE0B91508F415CDF0
:1042E000E92DF0E0E450F94C0C945336811491041C
:1042F00009F0CACA512C912C812C80E00E94C3176E
:10430000D092B104C092B00481E08093AD048FE0FC
:104310008A9DF0018B9DF00D1124E65DFC4F858197
:104320008093AB0451100EC08114910459F0808128
:1043300091819C0124503109213A310508F0CDCA00
:104340000E94F6048FE08A9DF0018B9DF00D1124F0
:10435000E65DFC4FC680D780C6019A9581159F41C6
:1043600010F420EED22299249394C60101978F3342
:104370009E4708F0912C8FE08A9DD0018B9DB00D57
:104380001124A65DBC4F1996ED91FC911A973097B8
:1043900031F01B966D917C9181E0099598229920CE
:1043A000B1F08FE08A9DF0018B9DF00D1124E65D48
:1043B000FC4F868197810E946B0B8093AC04C601F1
:1043C00048E06416710408F08BCA0E944E060E94F1
:1043D0004E128FCAB0E0A0E0E0EFF1E20C94FF359E
:1043E0008091CB01807F09F054C08091CA0188235D
:1043F00009F44FC0E091520589E0D82E809109055B
:104400008E1709F446C00E2F10E0ED9DF001112427
:10441000E65FFA4F8481882309F440C0D09EE00112
:10442000D19ED00D1124FE01E65FFA4F918180915B
:10443000C601981333C090818091C50198132EC096
:10444000858181112BC0E280F3808091C70190911A
:10445000C801E81AF90A60E085EC91E00E94650E57
:1044600065EC71E00E94CB0EE816F906B8F4809175
:10447000CB018F7080618093CB01C05FDA4F888160
:104480008F708061888385EC91E00E943D1A0E94C4
:104490006909CDB7DEB7E7E00C941B36F801319619
:1044A000E770ACCFA8E1B0E0E8E5F2E20C94F735B4
:1044B0008C0186E0F801DE01539601900D928A95F9
:1044C000E1F7D80114967C9014971596EC9085EC42
:1044D000A82E81E0B82E8091C90181112AC07110E7
:1044E00003C0FF24F3941CC0EE20F9F0C8010E9421
:1044F0002C0EF82E8823C9F089E0F801A5ECB1E074
:1045000001900D928A95E1F78091C901813031F4D3
:104510008091C5019091C6010E941F0E0E94EA2160
:104520008F2D6896EFE00C941336C8010E943D1A57
:10453000D8CFF80150806180C280D38060E085ECE4
:1045400091E00E94650EF090CA018091C7019091A0
:10455000C8014601881A990A60E085EC91E0FF20C5
:1045600009F428C10E94650E65EC71E00E94CB0E33
:104570008816990608F0D1C0772009F4B2CF80914F
:10458000CB01382F307F2091C601D80111969C9124
:104590001197311171C029131FC02091C5019C9141
:1045A00029131AC04091CC015091CD0117962D913D
:1045B0003C914217530781F4E11054C08F70806121
:1045C0008093CB0185EC91E00E943D1A8091CB0154
:1045D000F8018683F12CA4CFE11044C0662D852D0F
:1045E0000E942A03E82E882381F08091D00480FF66
:1045F000F1CF85EC91E00E943D1A89E0E5ECF1E015
:10460000DF011D928A95E9F7E5CF5B8A6C8A8B8979
:104610009C890E941F0E292F22952F70243058F458
:104620009F70223088F0992399F0F8019681907F4D
:1046300079F4FE2C75CF2A5F2F70223068F0C80104
:104640000E943D1AEF2CF5CF992311F0882389F3AE
:10465000805E883070F3F3CF803F58F3815F833002
:1046600070F7E7CF8091CB0181608093CB0180917F
:10467000D00481FDAFCFBDCF291320C02091C5014B
:104680009C9129131BC04091CC015091CD011796EC
:104690002D913C9118974217530781F4E1100EC0F9
:1046A00016968C93C8010E943D1A89E0F801A5EC8A
:1046B000B1E001900D928A95E1F732CFC8010E94D6
:1046C0002C0E882309F431CFEE2009F42ECF8091EF
:1046D000CB018032B8F02091C5013091C6013B87F3
:1046E0002A87DD86CC869091C9019E871F86888B9C
:1046F0008091CC019091CD019A8B898BCE010A9645
:104700000E943D1A89E0F801A5ECB1E001900D92FC
:104710008A95E1F70E94EA21E4CE8091CB01982F9F
:10472000907F09F466CF772009F4DBCE2091C60193
:10473000F801918129131AC02091C5019081291394
:1047400015C04091CC015091CD0127813085421791
:10475000530761F4E1100AC08683C8010E943D1A24
:1047600089E0D5011D928A95E9F7DACEC8010E9449
:104770002C0E882309F4D9CEEE2009F4D6CE8091F0
:10478000CB01803208F4BECF2091C5013091C60123
:104790003A832983DC82CB829091C9019D831E825A
:1047A0008F838091CC019091CD0199878887CE012C
:1047B0000196A6CF0E94650E65EC71E00E94CB0EBB
:1047C0008816990608F055C0772009F48ACEFE2C89
:1047D000EE2009F4AACE9091C601F80181819813C8
:1047E0003AC09091C5018081981335C02091CC01C9
:1047F0003091CD01878190852817390761F5A09008
:10480000C701B090C80160E085EC91E00E94650EA0
:104810008091D00482FD49CFCA18DB088091CB0477
:104820009091CC04C816D90608F03FCF8091CB01F7
:1048300080FD3BCF982F907F09F437CFD801169693
:104840008C931697903F09F42DCF982F907F905F0F
:104850008F70892B25CFC8010E942C0E811152CF59
:104860008091CB0181608093CB01C8010E943D1AE9
:1048700057CE89E0F50111928A95E9F751CEA2E170
:10488000B0E0E5E4F4E20C9402360A871B872C873B
:104890003D874E875F87688B798B8A8BCE010A961E
:1048A0000E94522281110CC089E0FE013A96DE017D
:1048B000119601900D928A95E1F78E8581110BC0BA
:1048C00019E08091520590910905891331C06296D3
:1048D000E4E00C941E362091090530E0C9010196F0
:1048E00087709927409152054817190699F099E069
:1048F000929FD001939FB00D1124A65FBA4FFE0185
:10490000319601900D929A95E1F7809309050E94E6
:104910006909D6CF0E94FE12109209051092520525
:1049200089E0E5ECF1E0DF011D928A95E9F7C8CF57
:10493000819FC0011124865F9A4F0E9452228823D2
:1049400031F28091520590E001968770992780930B
:104950005205B7CFEF92FF920F931F93CF93DF9340
:1049600080912804882361F0E091EF038DE0F82E18
:1049700080912804E81748F0109228041092EF0361
:10498000CDB7DEB7E6E00C941C36EE24E394EE0ED1
:10499000E092EF03CE2FD0E0EF9DF0011124E75D10
:1049A000FB4F84818823E9F087819085892B21F44E
:1049B00081859285019659F400811181228133818C
:1049C000448155816681778180850E943F24FC9EC9
:1049D000F001FD9EF00D1124E75DFB4F1482109253
:1049E0005305EE2DC5CF10929C0410929B0410929B
:1049F000380180919A04809399040E94ED060E94E8
:104A0000AA240895B0E0A0E0E8E0F5E20C94F535C2
:104A1000C091990497E0992E01E010E02DE0322E2C
:104A200034E0432E5524539480919A048C1309C08A
:104A30000E94AA240E94ED06CDB7DEB7E1E10C94F6
:104A40001136D0E0FE01EE0FFF1FEF56FB4F8081C5
:104A50009181989ED001999EB00D1124A051BC4F18
:104A600014962C911497211159C060902804E9E202
:104A7000F4E030E020E0812C5D01261508F04CC008
:104A8000E384F484D501CD90DC906FEF7FEF712C3F
:104A9000472D50E0DA01AA0FBB1FAC0DBD1D0D90D4
:104AA000BC91A02D109731F0EA16FB0609F4BA016B
:104AB0007394EECF6F3F7607A9F1D80102C0AA0F19
:104AC000BB1F6A95E2F78A2AB801072C02C0660F5D
:104AD000771F0A94E2F7AB0141505109841615067D
:104AE00001F5329EF001339EF00D1124E75DFB4F7E
:104AF000989ED001999EB00D1124A051BC4F1296E2
:104B00002D913C9113973087278344821082118224
:104B10009287818715965C920E94BF062196C3708A
:104B200083CF14822F5F3F4F3D96A7CFAEE1B0E019
:104B3000ECE9F5E20C94F4354B8B5C8B6D8B7E8B42
:104B40008F8B988F882349F08091A8019091A901BB
:104B500001969093A9018093A801888D81111092EC
:104B60005305188A198A1A8A86E0FE017396DE01B7
:104B70001A9601900D928A95E1F78091A30382FF26
:104B80001EC08091B5049091B604892BC1F00E949B
:104B9000EA042091CF013091D001821B930B209128
:104BA000B5043091B6048217930720F08091D101AB
:104BB00082FFE7C10E94450981110E94F6088E8597
:104BC000882389F061E0CE010A960E94650E6C018F
:104BD0008F8520E5C2162CE7D20689F4882329F1B7
:104BE00081E0809338010A851B852C853D854E85A3
:104BF0005F85688979898A890E943F24CDC031E523
:104C0000C3163CE7D30629F4882379F00E94F324E5
:104C1000EACF42E5C4164CE7D40639F4882329F0DC
:104C2000809138018111F2CFDBCF90EFE92E93E034
:104C3000F92E412CB12CA12C88248394912CBE01F7
:104C40006F5F7F4F7A8F698F22242394F701408111
:104C5000518166246A94762C20E0822F90E0FC013A
:104C6000EE0FFF1FE40FF51F608171816115710563
:104C700031F0C616D70609F43C012F5FEECF312C78
:104C8000FFEF6F167F0609F448C0F70144813090AA
:104C90003801832D411180E0F82FF1703F2EF7018C
:104CA000558086819F85992309F4F7C0332009F444
:104CB000F4C00091C9041091CA04511013C0A4019A
:104CC000062C01C0440F0A94EAF7842B8683809156
:104CD000ED039091EE038017910720F41093EE03FB
:104CE0000093ED03C40102C0880F991F2A95E2F7D3
:104CF0000197F70126812817190679F480919B0402
:104D000090919C04009709F44BC00E94CF040817AF
:104D1000190708F045C0F70124824328FFEFAF1AB6
:104D2000BF0A27E0E20EF11C38E0A316B10409F037
:104D30008DCF8F85882309F410C1442009F40DC15B
:104D40000E94EA0490939C0480939B048091280421
:104D5000883010F591E0980F9093280499E0FE01B7
:104D60003A96DE01119601900D929A95E1F74DE089
:104D7000849FC0011124875D9B4F29E0FE0131967D
:104D8000DC0101900D922A95E1F72FEF3FEFFC0136
:104D900032872187D486C3866E96E2E10C94103662
:104DA0008091990450919A04982FF0E0E0E08513E7
:104DB00014C090939904EE16FF0609F4AECF90E06C
:104DC000FC01EE0FFF1FEF56FB4FB182A082019650
:104DD0008370992780939A04A0CF682E712CF301D9
:104DE000EE0FFF1FEF56FB4F20813181F7E0F29F5E
:104DF000D001F39FB00D1124A051BC4F2D913C91D7
:104E000011973E8F2D8F40E020E030E0E32FF0E05F
:104E1000EE0FFF1F6D8D7E8DE60FF71F0081118154
:104E200001151105E1F0F7010190F081E02DFC8FF3
:104E3000EB8F20E005C00617170709F4432D2F5FFD
:104E4000E22FF0E0EE0FFF1F6B8D7C8DE60FF71F5A
:104E5000608171816115710571F73F5FD7CF442380
:104E6000C9F0F701231708F0FD012482EE16FF06B2
:104E700021F490939904342E50CF891305C0AE17B6
:104E8000BF0711F49F5F937093012F5F3F4F822FF5
:104E900083708DCFF0E0E0E0F7CF90E0511020C0BC
:104EA000B40102C0660F771F2A95E2F79B012150DB
:104EB00031092817390731F4442309F44CC0C501DE
:104EC0000E94BF06C401062C01C0880F0A94EAF7AD
:104ED000982F9095F701868189238683352C1DCFE5
:104EE000AC01062C02C0559547950A94E2F7BA0129
:104EF000617077279C012150310982239323892BEC
:104F000031F5672B21F1F70182819381892BE1F043
:104F1000E98DFA8D27E011922A95E9F70E94EA04BB
:104F2000282F8B839C8334E03D83F701828193811A
:104F3000782F8887998709811A813C8144E05E81B6
:104F40006F81892F0E943F24F7011582BBCFF42F78
:104F5000F1705F2EB7CF532CB5CF9091990480910B
:104F60009A04981729F00E940225411015CF3BCED4
:104F70000E94AA2410929C0410929B040E94ED06A9
:104F8000F4CF82E00E940E0A15CEA6E0B0E0EBEC72
:104F9000F7E20C9404369093460280934502811503
:104FA00020E2920730F40E9429182696E2E00C9441
:104FB000203680EF89838A830E94EA048160682F0B
:104FC0009C838B8349815A817C8181E090E00E949F
:104FD0009625EBCF0F931F93CF93DF938C01EB01BB
:104FE0006FE472E08C2F0E94B70E892BA1F48091A0
:104FF000D1049091D2040E94F90BDD27C95BDD4FEB
:105000008881F801128218828330F1F048F48130EF
:1050100059F0823081F0DF91CF911F910F91089567
:105020008430B9F08530B9F780914F0290915002E9
:10503000009789F306C08091510290915202009727
:1050400099F30E94C527E7CF8091530290915402B3
:10505000F6CF8091550290915602009791F72091DA
:105060004F023091500280915102909152022115CD
:105070003105F1F2009729F7C901E3CFA6E0B0E0CE
:10508000E4E4F8E20C9404369093460280934502DF
:10509000811520E2920730F40E9466192696E2E01C
:1050A0000C94203680EF89838A830E94EA04816011
:1050B000682F9C838B8349815A817C8181E091E0B8
:1050C0000E949625EBCFCF93DF93EC010E943E2800
:1050D0008091D1049091D2040E94F90BCE010E94DC
:1050E000C527DF91CF9108950F931F93CF93DF933F
:1050F0008C01862F6FE472E00E94B70E892BB1F409
:10510000C0914F02D0915002209781F0F801828126
:10511000833051F4CE010E946328CE010E9463289F
:10512000CE010E94632802C08430D0F7DF91CF9176
:105130001F910F9108950F931F93CF93DF938C01CD
:10514000EB016FE472E08C2F0E94B70E892B09F0FF
:105150005CC0FE01FF27D80112968C911297E95B83
:10516000FD4F8130B9F415969C9192FF02C0808367
:105170000AC090FFFCCF82E0808380915102909121
:1051800052020097B9F480914F029091500200971B
:10519000E1F110C08230B9F515968C9182FD28C0DE
:1051A00080FD0BC083E08083809153029091540274
:1051B000009701F10E943E2828C084E080838091FE
:1051C0005502909156020097A9F780914F02909155
:1051D00050020097F9F00E9463288091510290914B
:1051E0005202009739F780914F0290915002E2CF1E
:1051F00085E0808380914F0290915002009729F0C2
:105200000E946328F0CF86E08083DF91CF911F91C9
:105210000F9108958091510290915202B8CFA6E06B
:10522000B0E0E5E1F9E20C9402360E94EA048C0158
:105230008091DD019091DE018017910781F0198244
:105240001A820E94EA04682F49815A81792F80E0EE
:1052500090E00E9496251093DE010093DD012696D2
:10526000E4E00C941E361F920F920FB60F92112499
:105270002F933F934F935F936F937F938F939F935E
:10528000AF93BF93CF93DF93EF93FF93D091E90058
:10529000DF708091EC00C82FC17080FDC0E81092D3
:1052A000E9008091F000877F8093F00078940E945D
:1052B00025131092E9008091F00088608093F0003F
:1052C000CD2BCF70C093E900FF91EF91DF91CF918B
:1052D000BF91AF919F918F917F916F915F914F910E
:1052E0003F912F910F900FBE0F901F9018951F9216
:1052F0000F920FB60F9211242F933F934F935F930A
:105300006F937F938F939F93AF93BF93EF93FF938D
:105310008091E10082FF09C08091E20082FF05C018
:105320008091E1008B7F8093E1008091DA0080FF23
:1053300024C08091D80080FF20C08091DA008E7F49
:105340008093DA008091D90080FF9DC080E189BD03
:1053500082E189BD09B400FEFDCF81E08093FF04A6
:105360008091F204811109C00E9460030E9401042F
:105370008091E20084608093E2008091E10080FFF0
:1053800017C08091E20080FF13C08091E2008E7F01
:105390008093E2008091E20080618093E20080913E
:1053A000D80080628093D80019BC85E08093FF0408
:1053B0008091E10084FF2BC08091E20084FF27C030
:1053C00080E189BD82E189BD89B5982F917080FF08
:1053D000FBCF8091D8008F7D8093D8008091E10031
:1053E0008F7E8093E1008091E2008F7E8093E200C7
:1053F0008091E20081608093E20080910005882323
:1054000009F447C084E08093FF048091FF048091F9
:10541000E10083FF27C08091E20083FF23C08091D9
:10542000E100877F8093E10082E08093FF04109287
:1054300000058091E1008E7F8093E1008091E20081
:105440008E7F8093E2008091E20080618093E20091
:1054500042E060E080E00E94CF038091F00088602D
:105460008093F000FF91EF91BF91AF919F918F9149
:105470007F916F915F914F913F912F910F900FBE50
:105480000F901F90189519BC1092FF041092F2040F
:1054900074CF8091E30087FD93E09093FF04B5CF34
:1054A00078941F921FB61F9211248F939F93AF93EE
:1054B000BF938091EE049091EF04A091F004B0911D
:1054C000F1040196A11DB11D8093EE049093EF04A9
:1054D000A093F004B093F104BF91AF919F918F918D
:1054E0001F901FBE1F9018951F921FB61F92112468
:1054F0008F939F93AF93BF938091ED04811113C05D
:105500008091EE049091EF04A091F004B091F10429
:105510004196A11DB11D8093EE049093EF04A093DA
:10552000F004B093F104BF91AF919F918F911F90C0
:105530001FBE1F9018951F920F920FB60F92112445
:105540002F933F934F935F936F937F938F939F938B
:10555000AF93BF93EF93FF930E94370C811137C035
:105560008091C7038F5F8093C7038A3058F48230DD
:1055700008F03EC0813039F11092C7031092C60383
:1055800081E047C08A3009F447C08B30A9F70E94F8
:105590002D0C882389F35091C6034FB7F89480915E
:1055A000C50390E09C012F5F3F4F2F71332760911F
:1055B000C403621731F08C559C4FFC01508320933B
:1055C000C5034FBFD9CF0E942D0C8111D5CFFF91BC
:1055D000EF91BF91AF919F918F917F916F915F916B
:1055E0004F913F912F910F900FBE0F901F901895E4
:1055F0008091C60386958093C6030E942D0C882354
:1056000031F38091C60380688093C6038091340192
:105610008F5F80933401DBCF0E942D0C9091340179
:10562000882319F090FFA8CFD2CF90FDA5CFCFCF80
:10563000CDB7DEB7C054D1090FB6F894DEBF0FBEA8
:10564000CDBF85B7806885BF85B7806885BF84B7C3
:10565000877F84BF0FB6F894A89580916000886119
:1056600080936000109260000FBE80E890E00FB65B
:10567000F89480936100909361000FBE84ED97E0F1
:1056800090939D0180939C010E94AF070E94B50FEB
:105690000E94310F0E94910E0E9460030E9401043B
:1056A0008091E20084608093E20078948091FF040E
:1056B0008823A1F01091E9001F709091EC00892FD0
:1056C000817090FD80E8182B1092E9008091E8002D
:1056D00083FD0E9425131F701093E90082E084BDB2
:1056E00093E095BD9AEF97BD80936E0010920102F2
:1056F0001092020210920302109204020E948B0D7B
:10570000811102C00E94D0168091D80080618093E0
:10571000D8002AE12A95F1F700C08091D900182F0E
:10572000117080FD04C00E9460031092FF0410936A
:10573000E50484988C988FE891E00197F1F700C018
:1057400000008FB1829581708093E60480932501DB
:105750008091E50481110E9492348091250181118C
:105760002CC085E0EEE3F1E0DE01919601900D9210
:105770008A95E1F789A1809320018AA18093210174
:105780008BA1809322018CA1809323018DA1809312
:10579000240187E0E3E4F1E0DE01119601900D922F
:1057A0008A95E1F7FE013196A9E1B1E0CE010896B4
:1057B00021912D938E179F07D9F78091250195E0B0
:1057C000811190E09093100285E0891B80930F0275
:1057D00000E211E0D8018D918D018F3F11F00E9400
:1057E000D607B1E005321B07A9F709E111E030E265
:1057F000E32E31E0F32EF80181918F018F3F11F0FC
:105800000E94D607E016F106B1F78AE0E9E3F2E07C
:10581000DF01282F1D922A95E9F7E5E0F2E0DF018C
:105820001D928A95E9F790E080E00E949E36853EC1
:105830009E4F21F40E948B0D811163C065EE7EEFB7
:1058400090E080E00E94D23660E082E090E00E942A
:10585000B43681E08093110261E083E090E00E9421
:10586000B43660E074E184E090E00E94D23660E0FB
:1058700086E090E00E94B43660E087E090E00E940D
:10588000B43640E050E0BA0188E090E00E94C636AD
:1058900060E083E290E00E94B43660E08CE090E04B
:1058A0000E94B43660E08DE090E00E94B436198228
:1058B0001A821B821C821D821E821F82188648E06B
:1058C00050E067E170E0CE0101960E94A43640E00E
:1058D00050E0BA018FE190E00E94C63680E00E945D
:1058E0003C0D0E94D01640E050E0BA018FE090E0FD
:1058F0000E94C63640E050E0BA0183E190E00E9489
:10590000C63682E090E00E9496368093140284E0CE
:1059100090E00E949E369093A3038093A2030E947E
:10592000EE10EFEFF6E721E0E150F0402040E1F724
:1059300000C000000E94EE108091390280FF08C074
:105940006FEF7FEF90E080E00E94D2360E94BE04AD
:1059500083E090E00E9496360E94480A0E94040765
:105960000E94FE06809168008160809368008091AB
:105970006B00806280936B003FEF43ED80E331501A
:1059800040408040E1F700C000008FEF0E94690CAA
:105990000E94030C0E94030C80911302811103C02A
:1059A00085EF0E94690C80EF0E94690C80911302C0
:1059B000811103C084EF0E94690C81E0809313027F
:1059C00087EE0E94690C80911302811103C084EF5D
:1059D0000E94690C8091E504811102C00E949534F7
:1059E00086E291E09093EA048093E90489E392E0EF
:1059F000AAE0A80F2196AFAF219733243394222435
:105A00002394FE01BB96FBAFEAAF8E010F5F1F4FE1
:105A10009E012D5F3F4F3DAF2CAF8091FF0485303D
:105A200079F480E4F82E90E1E92E22E1D22E8091E3
:105A3000FF04853009F455C00E94FE120E947505CE
:105A40000E94EE10A5E1EA2EA2E0FA2EB9E3AB2EF9
:105A5000B2E0BB2E2FE132E0D501F70191918D919B
:105A60002E173F0709F471C09817C1F34090E50461
:105A7000F9E3CF2EF2E0DF2E912CD6018D906D014F
:105A8000F70151907F01581429F1712C6624639419
:105A90005824852D8621B1F04420A1F07CAA9DAA2E
:105AA0000E94EA049FAB8EAB28AE91E0882D862140
:105AB00009F490E099AF4CA95DA96EA97FA988ADC2
:105AC0000E9496257394660CF7E07F12E2CFF701EF
:105AD0003197808293942AE09212CFCF0E94ED07F3
:105AE00038C08091FF04843019F11092ED0488E1F0
:105AF00090E00FB6F894A895809360000FBEF092E6
:105B0000600083B7817F846083BF83B7816083BF78
:105B10007894889583B78E7F83BF0FB6F894A89545
:105B200080916000886180936000109260000FBED9
:105B30000E94EE10E9E3F2E08191811143C62196C3
:105B40009FAD21979E13F8CF72CF98138FCF0E94ED
:105B50000F298091E504882309F4BFC08091AE0429
:105B60009091AF04892B09F43EC04091A304509159
:105B7000A4046091A5047091A6042FB7F8948091B5
:105B8000EE049091EF04A091F004B091F1042FBFC6
:105B9000841B950BA60BB70B40919F045091A0045A
:105BA0006091A1047091A20484179507A607B70716
:105BB000D0F08091AE049091AF040E9466191092CB
:105BC000AF041092AE041092A3041092A404109299
:105BD000A5041092A60410929F041092A0041092A3
:105BE000A1041092A204C090E304D090E404C11474
:105BF000D10469F180911F02909120020E94CF048C
:105C00007C0189E0AAADBBAD1D928A95E9F7BE0182
:105C1000655D7F4FC6010E94CB0E8E159F05B8F4BF
:105C20002091E3043091E404C9019927287F3327A8
:105C3000232B09F016C1E4E0880F991FEA95E1F7DC
:105C4000875A9D4FFC01258122FF0E94B812809146
:105C50003801882301F180919B0490919C04009766
:105C6000D1F00E94CF042091ED033091EE0328176C
:105C7000390788F49091990480919A04981709F44F
:105C8000F3C00E9402251092EE031092ED031092D1
:105C90009C0410929B048091CE0480FF1EC08091D2
:105CA000370182FF1AC00E94EA042091E903309173
:105CB000EA03AC01421B530B2091350130913601B0
:105CC0004217530750F021E232E041E0BC018091DD
:105CD000EB039091EC030E948E1986E0EDEDF4E069
:105CE000D80101900D928A95E1F78090DE04D09062
:105CF000DF04E090E004C090E104F090E204109230
:105D0000DF041092E0041092E1041092E2048E2D60
:105D10008D2991F08091DB049091DC040E94CF04E6
:105D2000AC019091B204992309F4A7C0809132018B
:105D30008417150608F4AFC08F2D8C2991F080913F
:105D4000D9049091DA040E94CF04AC019091D70459
:105D5000992309F4DAC0809130018417150608F4FC
:105D6000E2C08091DE04881217C08091DF0488238E
:105D700011F08D1111C02091E004222311F0E212E4
:105D80000BC09091E204992311F09F1105C030914E
:105D9000E104332309F45FC50E948C0586E0F80115
:105DA000ADEDB4E001900D928A95E1F78091330258
:105DB00090E0019665E070E00E943F3680933302E8
:105DC000892B09F4EAC080916B008F7D80936B0072
:105DD0000E94750590913402891721F08093340256
:105DE0000E94DE048091FF04843009F016CE83E027
:105DF0008093E9008091E80082FF0FCE8091E80057
:105E000090E085FF0AC00E947F0370E2C72ED12C6C
:105E10007801882309F42FC191E08091E8008B7705
:105E20008093E800992309F4F8CDE0904302F090C4
:105E300044028981E114F10409F42BC18E3F09F079
:105E4000AEC18A81833020F08550833008F0A7C12D
:105E5000EA81EE3008F0A3C1F0E0E85FF84C0C9462
:105E6000533690E080E0EECE0E94AA2410929C046B
:105E700010929B040E94ED060ECF20913301FAE0B0
:105E80002F9F900111242417350708F055CF9F5FED
:105E90009093B20402C09F3FD1F7DD2059F00E94D9
:105EA000E1059FEF1D140CF491E0899F802D1124D2
:105EB0008093DF04EE2059F00E94E10591E01E146A
:105EC0000CF09FEF899F802D11248093E004809136
:105ED000DF04882309F430CF9090E004992009F47E
:105EE0002BCF0E944006882351F08093DF04892D38
:105EF0000E944006882331F08093E0041DCF309249
:105F0000DF04F5CF3092E00417CF209131018AE011
:105F1000289F900111242417350708F022CF9F5F96
:105F20009093D70402C09F3FD1F7CC2059F00E9434
:105F3000A8059FEF1C140CF491E0899F802D11247B
:105F40008093E104FF2059F00E94A80591E01F14FE
:105F50000CF09FEF899F802D11248093E2048091A3
:105F6000E104882309F4FDCEC090E204CC2009F4BA
:105F7000F8CE0E944006882351F08093E1048C2DD6
:105F80000E944006882331F08093E204EACE3092EA
:105F9000E104F5CF3092E204E4CE80916B008062A0
:105FA00080936B008BEE0E94690C8A3F09F010CF42
:105FB0000E94030C80932E020E94030C80932F02F8
:105FC0000E94030C30912E0290912B02392B4091AC
:105FD0002F0220912A022327277090913102942BBF
:105FE000292B282B39F130932A02942F990F940FE3
:105FF000282F220F820F232F207434FF26C0211157
:1060000003C0903809F097FF91E835FF24C037FDB1
:1060100003C0803809F087FF81E8377030932E0283
:10602000819580932F029195909330028DE292E0BA
:106030000E94670510922F021092300210923102D6
:106040001092320210922E02C3CE211102C097FF8D
:10605000DCCF9FE7DACF37FD02C087FFDECF8FE7C7
:10606000DCCF8091F100D7018D937D01B1E0CB1A97
:10607000D10809F4D1CE8091E80085FDF2CF80915E
:10608000E8008B778093E8000E947F03882399F3D0
:10609000C3CE8C3009F4C4C060F5843009F4A7C0C5
:1060A00050F4823009F46AC008F092C0813009F4DB
:1060B00061C08FEFB1C3863009F4AFC008F4A2C04D
:1060C0008B30B9F780919D0490919E04892B09F43F
:1060D00066C040E250E0B80182E00E949C0B3FEFB6
:1060E00041EE84E0315040408040E1F700C00000C4
:1060F0002DCC803109F4C3C088F58E3009F496C0E8
:1061000008F491C080919D0490919E04892B09F41C
:1061100046C0EC80F12C3DE1E316F10408F03FC0ED
:10612000CA80DB80DC24CD24DC245801E00EF11E83
:10613000C60184599C4FAE14BF0489F144E9C416CA
:10614000D10428F4D50114966C910E94B436BFEFA7
:10615000AB1ABB0AEFEFCE1ADE0AEACF823109F49E
:1061600093C008F48FC0833109F4B7C08E3F09F0A3
:10617000A0CF6ECE1A8289E08B8311C08A818230D3
:1061800009F46EC3833091F0813009F092CF0E9400
:10619000DE040E9459366B837C838D839E8340E2AC
:1061A00050E0B80182E00E949C0B37CC80919D04A6
:1061B00090919E04892B99F3FE01339683E492E03B
:1061C000D5012D915D0121938A179B07C9F7E7CF70
:1061D0008A81823009F06DCF6B817C818D819E81B7
:1061E0000E94593687E290E00E94B436D8CF4C81A5
:1061F0006B818A810E94A40D9827892798279E8306
:106200008D83CDCF2D813E813227232732274C81AC
:106210006B818A810E94650DC2CF0E944016BFCF5C
:1062200080E18A83BCCF1A8284E9A6CFEC80F12C6E
:10623000BDE1EB16F10408F0B2CFCA80DB80DC24AC
:10624000CD24DC245801E00EF11EC60184599C4F78
:10625000EA14FB0409F4A3CFE4E9CE16D10460F4F8
:106260000E949636D50114968C93FFEFCF1ADF0A61
:106270002FEFA21AB20AE9CFF5011482F6CF0E94DD
:10628000550D8DCF84E0CDCFEC80F12CFDE1EF16E4
:10629000F10408F084CFCA80DB80DC24CD24DC2428
:1062A0005801E00EF11EC6018896AE14BF0409F431
:1062B00076CF20E3C21622E0D20660F40E94963622
:1062C000D50114968C93FFEFCF1ADF0A2FEFA21A95
:1062D000B20AE9CFF5011482F6CFCC80D12C3DE192
:1062E000C316D10408F05BCFEA80FB80FE24EF24C4
:1062F000FE2440E3E41642E0F40608F050CF80E3C9
:1063000092E08E199F098C159D0508F448CF37013E
:1063100088E2680E711C80919D0490919E04270173
:106320004C0C5D1C892BB9F5570191E0A922BB24C7
:10633000E0FE0DC0C70187960E9496369D81892791
:106340009827892781159C4711F48FEF8D8346018B
:1063500040FE1AC0B1E08B1A9108E5E0F0E0EC0FC6
:10636000FD1FE80DF91DFFAFEEAFC3018C0D9D1DA4
:106370000E949636AEADBFAD9C9181159C4721F42D
:106380008FEFEEADFFAD8083F801EA0DFB1D2FEF1F
:10639000A814B90410F068011BC09481858181158F
:1063A0009C4711F42483258342E0A40EB11C32964D
:1063B000EFCFA0E3EA16A2E0FA0620F4F60164812A
:1063C0000E94B436FFEFCF1ADF0A2FEFE21AF20A6B
:1063D000C70188964E145F0461F7E1CE88E0EAE4D5
:1063E000F1E0DE01919601900D928A95E1F780E24D
:1063F000D8011D928A95E9F786E0898388E0FE013D
:10640000B196DE01159601900D928A95E1F7C7CEFF
:1064100088E989833A821B821C82C1CE8C81682FD5
:1064200070E0762F66278B81860F972F911D092E9E
:10643000000CAA0BBB0B65E0880F991FAA1FBB1F9E
:106440006A95D1F7AC01BD01405E5F4F6F4F7F4F42
:10645000481759076A077B0708F4A1CE8839E1E09D
:106460009E07A105B10508F09ACE4939F1E05F0712
:106470006105710520F048E951E060E070E0481BDB
:10648000590BBC0163577E4FC8010E94603687CE0E
:106490004AE150E06FEF70E0CE0107960E947F3630
:1064A00080919D048983EA821B821C8285E08D8312
:1064B0008E8375CE81E090E09093440280934302F6
:1064C00082E390E090933802809337020E94EA04BE
:1064D000909336028093350262CEEF2861F1F090FE
:1064E0003902E0903E0280913502909136020E947E
:1064F000CF048536910540F1E5FE26C0F0FE24C0AC
:106500000E94EA049093360280933502809137020C
:106510009091380201979093380280933702892B2B
:1065200051F4109244021092430281E090E0909363
:106530009E0480939D0480919D04898380914302F1
:106540008A838091370218CE82E390E090933802DC
:1065500080933702F0CF10929E0410929D041FCEBC
:10656000EB80FC8040E250E06FEF70E0C8010E94D9
:106570007F3625E233E0A1E2B4E090E080E0AC01B8
:106580004E5F5F4F4132510508F009CEF901659128
:106590007491E616F70630F4800F911FFC017183A9
:1065A0006083CA01245F3F4FA217B30741F7F7CDBD
:1065B0004B815C8185E293E021E234E0FC0165914E
:1065C00074914617570709F418C10C962817390714
:1065D000A9F76FCD2B813C8145E2E42E43E0F42EF8
:1065E00081E294E0F701459154912417350709F4AD
:1065F00015C1FCE0EF0EF11C8E159F0599F7CC2418
:10660000CA94DC2C26C10E94EE15C9CDEB81E7307F
:1066100008F0C5CDF0E0EA5EF84C0C9453368EE1FC
:10662000ACADBDAD1D928A95E9F788E089838A8378
:10663000A3CD8C819AE0D92E7E01B1E2EB0EF11C44
:10664000F7012D2D11922A95E9F7B7010E94B70E97
:106650008983F701DE01129601900D92DA94E1F739
:106660009ECDFC808AE0FE013596DE019196019078
:106670000D928A95E1F789A19AA10E94C7079AA372
:1066800089A38BA19CA10E94C7079CA38BA38DA16A
:106690009EA10E94C7079EA38DA38FA198A50E94CB
:1066A000C70798A78FA337E08FEF3F1568F04AE040
:1066B000F49EB001112464587D4F4AE050E0CE01B1
:1066C00081960E94D83680E089830E94AF0767CD0B
:1066D0006C812AE0CE018196DC01E22F1D92EA95C1
:1066E000E9F7683008F047C0629FB0011124645395
:1066F0007D4F4AE050E00E94863680E089838AE040
:10670000FE01B196DE0112967ECEFC808AE0FE018B
:106710003596DE01919601900D928A95E1F789A553
:106720009AA50E94C7079AA789A7F7E08FEFFF15E0
:1067300068F02AE0F29EB001112464537D4F4AE0D4
:1067400050E0CE0181960E94D83680E089830E9475
:10675000B50F25CD6C812AE0CE018196DC01E22FB8
:106760001D92EA95E9F7683030F4629FB001112478
:10677000645E7C4FBECF8FEFC1CFFC808AE0FE010C
:106780003596DE01919601900D928A95E1F78BA1E5
:106790009CA10E94C7079CA38BA3F7E08FEFFF1576
:1067A00068F02AE0F29EB0011124645E7C4F4AE05A
:1067B00050E0CE0181960E94D83680E089830E9405
:1067C000310FEDCC8091FE04882309F430C9E9BC77
:1067D000D9BC09B400FEFDCF8091D8008F7D809395
:1067E000D8008091E00082608093E0008091E0001A
:1067F00081FDFCCF0E94FE121AC9FC01369625913C
:1068000034912115310509F454CC4FE150E0BE011B
:106810006E5F7F4FF90109958983C1CCF7013896E6
:10682000259134912115310509F4E9CE4CE150E070
:10683000BE016B5F7F4FC701F90109956C01892B80
:1068400041F4F7013A9685919491009711F0FC017B
:106850000995C982A4CC822B892B09F49FCA9CCAB2
:1068600087E290E00E9496361B821C821D8220CE19
:106870008EE1669B02C08150E1F7669BFECF0895D2
:10688000769880E28A95F1F7769A0895FC013BE0CC
:106890003A95F1F798E020E080E031E040E14A9558
:1068A000F1F7880F669B02C08160232742E04A957A
:1068B000F1F7000040E14A95F1F7915079F790E146
:1068C0009A95F1F79CB132E03A95F1F7000040E17A
:1068D0004A95F1F796FB992790F992272081920F1C
:1068E00090830895A1E0B0E0E8E7F4E30C9400366B
:1068F00019828C017C01E60EF11C0E151F0541F476
:1069000081E09981911180E02196E6E00C941C369B
:106910000E943834CE0101960E944634F8018193DA
:106920008F01EBCF6E9A769A08956E98769AEE9ACA
:10693000EAE6F0E080818F7C808308956150770BD8
:1069400091E001C0990F6A95EAF720E031E09111DA
:1069500008C0222391F0769A80E28A95F1F7769822
:106960000895492F482339F0769A232740E24A9523
:10697000F1F79695ECCF7698F9CF7698EDCFFF9218
:106980000F931F93CF93DF93EC018C01060F111D22
:10699000C017D10729F4CDB7DEB7E5E00C941D365A
:1069A000F9900E94403468E08F2D0E949E34F0CF11
:1069B0001F920F920FB60F9211240F931F932F93D4
:1069C0003F934F935F936F937F938F939F93AF9377
:1069D000BF93EF93FF93CF93DF930F92CDB7DEB7C3
:1069E00019820E943834CE0101960E944634082F45
:1069F000069506950695282F22952570902F95705F
:106A0000290F922F937026952695920F98279770AD
:106A10008981982B09F05CC0043008F059C080E1EE
:106A20008A95F1F7769A6E9A82E08A95F1F700C01E
:106A3000769888E0089F80011124D801AF5FBE4F8F
:106A40001696ED91FC9117973097A9F060918B0104
:106A500070918C0114962D913C911597260F371F3C
:106A600011968D919C911297680F791F13964C91F6
:106A700013978C910995F801EF5FFE4F63816623B0
:106A800051F020918B0130918C0184819581820F8E
:106A9000931F0E94BF340E94403480E18A95F1F731
:106AA00076986E98769A80E18A95F1F7F801EF5F13
:106AB000FE4F6081662351F020918B0130918C0153
:106AC00081819281820F931F0E9472340E94383418
:106AD0000F90DF91CF91FF91EF91BF91AF919F9177
:106AE0008F917F916F915F914F913F912F911F9166
:106AF0000F910F900FBE0F901F9018950F931F933B
:106B0000CF93DF93EC0104970CF04CC0F8946E9A8D
:106B1000769885E08A95F1F700009C2F9695957000
:106B20008C2F8570980F892F83709695969523E00A
:106B3000CC0FDD1F2A95E1F7980F8E01092B0E94DB
:106B4000403400C068E0802F0E949E3480E18A9526
:106B5000F1F76E98769A669B1EC087E090E0669982
:106B60001CC0FE01EF5FFE4F63816623F9F02091A8
:106B70008B0130918C0184819581820F931F0E943B
:106B80007234811113C06E9A769A7894DF91CF9106
:106B90001F910F91089500C0DECF019729F46E9ADE
:106BA000769A789480E0F2CF00C0D9CF0E94383432
:106BB00080E28A95F1F776986E9A80E18A95F1F7EE
:106BC000CF5FDE4F6881662351F020918B013091B9
:106BD0008C0189819A81820F931F0E94BF340E9489
:106BE0004034789481E0D2CF2F923F924F925F92BF
:106BF0006F927F928F929F92AF92BF92CF92DF92CD
:106C0000EF92FF920F931F93CF93DF93CDB7DEB731
:106C1000CA1BDB0B0FB6F894DEBF0FBECDBF0994C5
:106C20002A88398848885F846E847D848C849B841C
:106C3000AA84B984C884DF80EE80FD800C811B812A
:106C4000AA81B981CE0FD11D0FB6F894DEBF0FBE59
:106C5000CDBFED010895AA1BBB1B51E107C0AA1FC0
:106C6000BB1FA617B70710F0A61BB70B881F991FED
:106C70005A95A9F780959095BC01CD01089597FB91
:106C8000072E16F4009407D077FD09D00E942B360A
:106C900007FC05D03EF4909581959F4F089570951F
:106CA00061957F4F0895EE0FFF1F0590F491E02D41
:106CB00009946927962769277827872778270895D1
:106CC000FB01DC0102C005900D9241505040D8F705
:106CD0000895FB01DC0104C08D910190801921F41D
:106CE00041505040C8F7881B990B0895FB01DC0107
:106CF00002C001900D9241505040D8F70895DC0138
:106D000001C06D9341505040E0F70895DC01CB0184
:106D1000FC01F999FECF06C0F2BDE1BDF89A3196AB
:106D200000B40D9241505040B8F70895F999FECF44
:106D300092BD81BDF89A992780B50895A8E1B0E089
:106D400042E050E00C948836DC01A40FB51F41509E
:106D5000504048F0CB01840F951F2E910E94B5360C
:106D600041505040D0F70895262FF999FECF92BD9B
:106D700081BDF89A019700B4021639F01FBA20BD00
:106D80000FB6F894FA9AF99A0FBE08950396272F32
:106D90000E94B5360E94B436252F0E94B536242FA6
:106DA0000C94B5360196272F0E94B5360C94B43654
:106DB000DC01CB0103C02D910E94E33641505040CD
:106DC000D0F70895262FF999FECF1FBA92BD81BD45
:106DD00020BD0FB6F894FA9AF99A0FBE019608955D
:106DE000F894FFCF06142E14DC152E14DC15611454
:106DF0008214DC158B1598152A1E2A1E5F1E5F1E35
:106E0000281F441F851E851E491FB61FC71FC71F89
:106E1000EE3108320E32CF30CF3048325A326D3236
:106E2000AB32B032D832EA32033306330F33193380
:0A6E3000313368338533AA33BD33D4
:106E3A000100000001000000000000000501000040
:106E4A00000406000000000000F5F6F73133323680
:106E5A00919094669701BB04E50BBA04DE0BD70B3D
:106E6A005001140101AF0001011E0A280801919086
:106E7A00946697323331F7F6F53698CC693A4B2D4A
:106E8A00DFEA818283E200E900EA00B500B600B7D2
:106E9A0000CD008301CC008A0192019401210223D2
:106EAA000224022502260227022A02B300B4006F36
:106EBA000070009F01CB019F02A002F20144227BD5
:0C6ECA0049012701AC00BF04D804F80403
:00000001FF
